:100000000C94B8010C94CE320C94FB320C94E001A9
:100010000C94E0010C94E0010C94E0010C94E001DC
:100020000C94E0010C94E0010C94E0010C94CB06DC
:100030000C94E0010C94E0010C94E0010C94E001BC
:100040000C94DA310C94E0010C9441060C947D067A
:100050000C94E0010C94E0010C94E0010C94E0019C
:100060000C94E0010C94E001084AD73B3BCE016EB2
:1000700084BCBFFDC12F3D6C74319ABD56833DDAFF
:100080003D00C77F11BED9E4BB4C3E916BAAAABE0E
:10009000000000803F05A84CCDB2D44EB93836A937
:1000A000020C50B9918688083CA6AAAA2ABE000074
:1000B00000803F0664EC1B3C04BC163E3BE5B93CAB
:1000C000C93C37C29E5A3D660498083EEA69AAAA0E
:1000D0003E000000803F2020BF0020BF00BF007C0A
:1000E0002020202020202020202020202020202010
:1000F00020202000C8202020202020202020202078
:1001000020C900C8202020202020202020202020BE
:10011000C97C00D820202020202020202020202042
:10012000D97C00C820202020202020202020202032
:10013000C97C00C820202020202020202020202032
:10014000C97C002070696E31002061727373690090
:10015000207265766F006D696E6F706F736400203A
:1001600020202020BABBBCBDBE7C2020202020CA7D
:10017000CBCCCDCE7C00626F6F74696E67207570DA
:100180003AEDF2F2F2F2F2F2F2F3006261747465A7
:100190007279207761726E696E6720007478706979
:1001A000642076616C756573006261726F2074659E
:1001B0006D700074656D70646973702000616374A4
:1001C0006976652000706173736976650075617684
:1001D00074616C6B20007365747570207363726555
:1001E000656E7C7C7C004368617220446F6E650A9A
:1001F00000526561647920666F7220466F6E740AE2
:1002000000557064617465204368617253657400C1
:1002100000407A10F35A00A0724E18090010A5D4BD
:10022000E80000E87648170000E40B54020000CA1A
:100230009A3B000000E1F505000080969800000060
:1002400040420F000000A0860100000010270000BF
:100250000000E803000000006400000000000A0045
:10026000000000000100000000002C76D888DC6748
:100270004F0823DFC1DFAE59E1B1B796E5E3E453A0
:10028000C63AE651997696E8E6C28426EB898C9BBD
:1002900062ED407C6FFCEFBC9C9F40F2BAA56FA55D
:1002A000F490055A2AF75C936B6CF9676DC11BFCDF
:1002B000E0E40D47FEF520E6B500D0ED902E0300FA
:1002C000943577050080841E080000204E0A000047
:1002D00000C80C333333330F986E12831141EF8D06
:1002E0002114893BE65516CFFEE6DB18D1844B3846
:1002F0001BF77C1D901DA4BBE424203284725E2277
:100300008100C9F124ECA1E53D276E616E00696EA4
:10031000660000000000240027002A000000000002
:10032000250028002B0000000000230026002900E3
:10033000040404040404040402020202020203038B
:100340000303030301020408102040800102040893
:100350001020010204081020000000070002010024
:100360000003040600000000000000004C04120816
:1003700011241FBECFEFD8E0DEBFCDBF13E0A0E059
:10038000B1E0EEE8F0E702C005900D92AE3FB10794
:10039000D9F716E0AEEFB3E001C01D92A53BB1075F
:1003A000E1F713E0C0E7D3E004C02297FE010E940A
:1003B0004138CC36D107C9F70E940A340C9445382D
:1003C0000C940000FA01AA27283051F1203181F164
:1003D000E8946F936E7F6E5F7F4F8F4F9F4FAF4F4D
:1003E000B1E03ED0B4E03CD0670F781F891F9A1F60
:1003F000A11D680F791F8A1F911DA11D6A0F711D14
:10040000811D911DA11D20D009F468943F912AE01F
:10041000269F11243019305D3193DEF6CF01089507
:10042000462F4770405D4193B3E00FD0C9F7F6CF38
:10043000462F4F70405D4A3318F0495D31FD405200
:10044000419302D0A9F7EACFB4E0A6959795879596
:1004500077956795BA95C9F7009761057105089575
:100460009B01AC010A2E0694579547953795279521
:10047000BA95C9F7620F731F841F951FA01D0895B9
:10048000283008F027E03327DA01990F311D87FD66
:10049000916000966105710539F432602E5F3D93DD
:1004A00030E32A95E1F708959F3F30F080387105D9
:1004B000610509F03C5F3C5F3D93913008F0806836
:1004C000911DDF93CF931F930F93FF92EF92192FFC
:1004D000987F9695E92F96959695E90FFF27E6590F
:1004E000FD4F99273327EE24FF24A701E70105904C
:1004F0000894079428F4360FE71EF81E491F511D73
:10050000660F771F881F991F0694A1F7059007941F
:1005100028F4E70EF81E491F561FC11D770F881FCC
:10052000991F661F0694A1F70590079428F4F80E0A
:10053000491F561FC71FD11D880F991F661F771FA0
:100540000694A1F70590079420F4490F561FC71F82
:10055000D81F990F661F771F881F0694A9F78491EB
:100560001095177041F0D695C79557954795F79414
:10057000E7941A95C1F7E0E1F2E0689415901591BF
:1005800035916591959105907FE27395E118F10A97
:10059000430B560BC90BD009C0F7E10CF11E431FEA
:1005A000561FC91FD01D7EF4703311F48A95E6CF13
:1005B000E894015030F0080F0AF40027021708F4FD
:1005C000202F2395022F7A3328F079E37D932A9503
:1005D000E9F710C07D932A9589F60694979567955B
:1005E000379517951794E118F10A430B560BC90B71
:1005F000D00998F023957E9173957A3308F070E3D3
:100600007C932013B8F77E9170617D9330F08395D1
:1006100071E37D9370E32A95E1F71124EF90FF9049
:100620000F911F91CF91DF91992787FD90950895A4
:10063000CF93DF93BC018230910510F462E070E04B
:10064000A091B306B091B406ED0140E050E0E0E0C7
:10065000F0E021C0888199818617970769F48A8123
:100660009B81309719F09383828304C09093B406E2
:100670008093B306FE0134C06817790738F441153A
:10068000510519F08417950708F4AC01FE018A8121
:100690009B819C01E9012097E9F641155105A9F1DB
:1006A000CA01861B970B049708F4BA01E0E0F0E05A
:1006B0002AC08D919C91119784179507F9F46417BE
:1006C000750781F412968D919C911397309719F0CC
:1006D0009383828304C09093B4068093B306FD0194
:1006E00032964CC0CA01861B970BFD01E80FF91F1B
:1006F0006193719302978D939C9340C0FD01828119
:1007000093819C01D9011097A1F68091B106909137
:10071000B206892B41F480919F029091A0029093A0
:10072000B2068093B1064091A1025091A2024115F8
:10073000510541F44DB75EB780919D0290919E02A4
:10074000481B590B2091B1063091B206CA01821B99
:10075000930B8617970780F0AB014E5F5F4F8417AE
:10076000950750F0420F531F5093B2064093B106C5
:10077000F9016193719302C0E0E0F0E0CF01DF91F5
:10078000CF910895CF93DF93009709F450C0EC0107
:1007900022971B821A82A091B306B091B4061097DB
:1007A00009F140E050E0AC17BD0708F1BB83AA8314
:1007B000FE0121913191E20FF31FAE17BF0779F4CB
:1007C0008D919C911197280F391F2E5F3F4F3983D0
:1007D000288312968D919C9113979B838A83411550
:1007E000510571F4D093B406C093B30620C012969D
:1007F0008D919C911397AD01009711F0DC01D3CF3F
:10080000FA01D383C28321913191E20FF31FCE17F6
:10081000DF0769F488819981280F391F2E5F3F4FC8
:10082000FA01318320838A819B8193838283DF91C4
:10083000CF910895FC010590615070400110D8F7E8
:10084000809590958E0F9F1F0895FC016150704018
:1008500001900110D8F7809590958E0F9F1F0895F5
:100860006EBD0DB407FEFDCF8EB508958DE061E03D
:100870000E9428338BE061E00E9428338CE060E026
:100880000E9428338AE061E00E9428331CBC80E586
:100890008CBD8DB58EB508958EEF93E00E94360421
:1008A0000895FC011382128288EE93E0A0E0B0E08C
:1008B00084839583A683B78384EB92E091838083BE
:1008C0000895FC018089803419F421E030E002C0F1
:1008D00020E030E0C9010895FC01818990E008958D
:1008E000FC016487458766874787089580E090E02C
:1008F000089580E090E0089580E090E008950895E4
:10090000EF92FF921F93CF93DF93162F7A0186E029
:1009100060E00E9467338EEF93E060E00E94300455
:100920008EEF93E060E00E9430048EEF93E069E088
:100930000E9430048EEF93E0612F0E943004C0E0EB
:10094000D0E0F701EC0FFD1F10818EEF93E06AE01D
:100950000E9430048EEF93E06C2F0E9430048EEFE3
:1009600093E06BE00E9430048EEF93E0612F0E94D1
:1009700030042196C633D10521F78EEF93E068E06D
:100980000E9430048EEF93E060EA0E9430048EEF04
:1009900093E060EA0E94300485FDF9CF8EEF93E08A
:1009A00060E00E9430048EEF93E06CE00E9430041F
:1009B00086E061E00E946733DF91CF911F91FF9045
:1009C000EF9008951F93CF93DF93EC01162F86E0ED
:1009D00060E00E9467338EEF93E060E00E94300495
:1009E000112319F0113059F404C08EEF93E0688997
:1009F00004C068896C618EEF93E00E94300486E049
:100A000061E00E946733DF91CF911F910895EF92CB
:100A1000FF920F931F938EE1489F70011124E60E01
:100A2000F11C86E060E00E9467330EEF13E0C8011E
:100A300065E00E943004C8016F2D0E943004C80197
:100A400066E00E943004C8016E2D0E9430041F91A0
:100A50000F91FF90EF900895EF92FF920F931F93E5
:100A60007C010EEF13E0C80167E00E943004C8016A
:100A70006FEF0E94300486E061E00E946733F70167
:100A800087858F5F87871F910F91FF90EF90089563
:100A9000EF92FF920F931F93FC01E7848EE1E89E93
:100AA000700111248685E80EF11C86E060E00E944A
:100AB00067330EEF13E0C80164E00E943004C80100
:100AC00063E00E943004C80165E00E943004C80160
:100AD0006F2D0E943004C80166E00E943004C801F6
:100AE0006E2D0E9430041F910F91FF90EF9008959A
:100AF0001F93CF93DF93EC01162F6C3731F40E94D4
:100B00002C05CE010E9448050AC08EEF93E067E0F5
:100B10000E9430048EEF93E0612F0E94300481E048
:100B200090E0DF91CF911F9108950F931F9386E07E
:100B300060E00E9467330EEF13E0C80164E00E949A
:100B40003004C80164E00E94300486E061E00E9445
:100B500067331F910F9108951F93CF93DF93EC019B
:100B6000188A16E0198B81EA96E060E973E00E942A
:100B70003A31813049F480E4888B88E0898B86E0C3
:100B800060E00E94673302C0188A198B86E060E03B
:100B90000E946733DF91CF911F9108950F931F93A8
:100BA000CF93DF93EC0186E061E00E94283382E07E
:100BB00060E00E94283382E061E00E946733CE014A
:100BC0000E94AC0586E060E00E9467338EEF93E000
:100BD0006CEE0E9430048EEF93E06FEF0E943004C1
:100BE000182F8EEF93E060E00E9430046889626005
:100BF0008EEF93E00E94300462E370E080E090E0CA
:100C00000E9430328EEF93E06CE60E9430041F7E2B
:100C10008EEF93E0612F0E9430048889803419F0B0
:100C20000DE010E002C000E110E01092000410920C
:100C3000FF0317C06091FF0370910004605F8EEFA7
:100C400093E00E9430048EEF93E069E00E9430044C
:100C50008091FF039091000401969093000480938B
:100C6000FF038091FF03909100048017910714F314
:100C7000CE0161E00E94E204DF91CF911F910F91BC
:100C800008951F920F920FB60F9211242F933F9346
:100C90004F938F939F93EF93FF934091C6002091C2
:100CA0009006309191062F5F3F4F8091940690916E
:100CB0009506282339238091920690919306281750
:100CC000390779F08091900690919106E09196060F
:100CD000F0919706E80FF91F408330939106209317
:100CE0009006FF91EF919F918F914F913F912F919E
:100CF0000F900FBE0F901F9018951F920F920FB676
:100D00000F9211242F933F938F939F93EF93FF9311
:100D100020919A0630919B068091980690919906B1
:100D200028173907E9F080919A0690919B06E09187
:100D30009E06F0919F06E80FF91F80818093C60000
:100D400080919A0690919B06019620919C06309185
:100D50009D068223932390939B0680939A0610C04E
:100D6000209198063091990680919A0690919B0661
:100D70002817390729F48091C1008F7D8093C10025
:100D8000FF91EF919F918F913F912F910F900FBE07
:100D90000F901F9018951F920F920FB60F9211246B
:100DA0008F939F938091C1049091C204892B51F03D
:100DB0008091C3049091C40401969093C4048093DD
:100DC000C30409C08091C5049091C6040196909314
:100DD000C6048093C5049F918F910F900FBE0F9012
:100DE0001F901895CF93DF93482FEB018091260633
:100DF000833009F45DC0843028F48130C1F0823042
:100E000058F50AC0853009F4D2C0853008F4A8C06E
:100E1000863009F0F2C0E9C04C3309F0EEC081E041
:100E200080932606488384EB80932506E6C0842FB2
:100E300090E0E0912506F0E0E827F927EE53FD4F1A
:100E4000208120932506887F9070809741F582E06D
:100E500080932606498329C0242F30E0E09125069F
:100E6000F0E0E227F327EE53FD4F808180932506C3
:100E7000809124068F5F80932406823018F43B8390
:100E80002A83BBC0922F88272A813B81820F931F20
:100E90009B838A830A978F3F910521F018F0109267
:100EA0002606ABC083E08093260610922406A5C0D8
:100EB000E42FF0E08091250690E0E827F927EE5333
:100EC000FD4F808180932506609124066F5F6093BB
:100ED0002406623089F0633020F4613009F08DC05F
:100EE00006C0633091F0643009F087C022C0842FBF
:100EF00090E0A0E0B0E018C0242F30E040E050E0E7
:100F0000542F432F322F222707C0242F30E040E0F8
:100F100050E0A901332722278C819D81AE81BF81BA
:100F2000820F931FA41FB51F8C839D83AE83BF8345
:100F300064C0242F30E040E050E0522F4427332794
:100F400022278C819D81AE81BF81820F931FA41FB8
:100F5000B51F8C839D83AE83BF8360932606A5CF88
:100F6000242F30E0E0912506F0E0E227F327EE534E
:100F7000FD4F808180932506809124068F5F8093AA
:100F80002406813019F08230C1F503C039872887E3
:100F900034C0922F882728853985280F391F398733
:100FA00028878A819B810A97F1F085E07CCFE42F26
:100FB000F0E08091250690E0E827F927EE53FD4FF9
:100FC000808180932506209124062F5F209324069C
:100FD00030E0FB01E20FF31F41878A819B810A9772
:100FE0002817390750F086E05ECFC75FDE4F488391
:100FF000C950D14087E0809326068091260687302D
:1010000069F410922606C75FDE4F9091250688810D
:10101000C950D140981711F48A8101C080E0DF9156
:10102000CF9108958F92AF92CF92EF92FF920F934C
:101030001F9387E894E060E045EC50E024EC30E05A
:1010400000EC10E0B1ECEB2EF12CCC24C394A8E919
:10105000AA2EF0E28F2E0E94AA2A84EA94E00E942F
:1010600051041092B7041092B8041092B90410926F
:10107000BA041092BB041092BC041092BD041092EA
:10108000BE041092C0041092BF041092B6041F91C7
:101090000F91FF90EF90CF90AF908F900895AF9207
:1010A000BF92CF92DF92EF92FF920F931F93E09047
:1010B0008C06F0908D0600918E0610918F068FE5BC
:1010C00090E0A0E0B0E0E80EF91E0A1F1B1F0E948E
:1010D00022326E157F058007910708F44EC0A0905C
:1010E000EC04B090ED04C090EE04D090EF04C60183
:1010F000B50120E030E040E85FE30E94AA36181610
:1011000094F5E0904406F090450600914606109153
:1011100047060E94223220918C0630918D06409124
:101120008E0650918F06621B730B840B950B0E94E9
:1011300080359B01AC01C601B5010E94B53620E0A7
:1011400030E04AE754E40E94E7349B01AC01C80157
:10115000B7010E941A346093440670934506809349
:101160004606909347060E94223260938C06709345
:101170008D0680938E0690938F061F910F91FF909E
:10118000EF90DF90CF90BF90AF900895DF93CF9313
:1011900000D000D0CDB7DEB7FB01E80FF91F6285A4
:1011A00083859485258569838A839B832C83492F36
:1011B0005C81782FCA010F900F900F900F90CF9104
:1011C000DF910895AF92BF92DF92EF92FF920F935B
:1011D0001F93CF93DF938C018091270680FDE4C09D
:1011E000F801F08087E894E06F2D0E948B2BE801D6
:1011F000C75FDE4FEF2DF0E0EE53FD4F8081888317
:10120000F801F18087E894E06F2D0E948B2BEF2D81
:10121000F0E0888190E0E827F927EE53FD4F8081C8
:101220008883F801F28087E894E06F2D0E948B2B71
:10123000EF2DF0E0888190E0E827F927EE53FD4F8D
:1012400080818883F801F38087E894E06F2D0E9405
:101250008B2BEF2DF0E0888190E0E827F927EE5303
:10126000FD4F80818883F801F48087E894E06F2D3A
:101270000E948B2BEF2DF0E0888190E0E827F92782
:10128000EE53FD4F80818883F801248135814681AA
:101290005781232F342F452F5527F22E87E894E0CE
:1012A000622F0E948B2BEF2DF0E0888190E0E827E1
:1012B000F927EE53FD4F80818883F8012481358121
:1012C000468157819A0144275527F22E87E894E0FA
:1012D000622F0E948B2BEF2DF0E0888190E0E827B1
:1012E000F927EE53FD4F80818883F80124813581F1
:1012F00046815781252F332744275527F22E87E82B
:1013000094E0622F0E948B2BEF2DF0E0888190E01B
:10131000E827F927EE53FD4F8081888387E894E022
:1013200060E00E948B2BE881F0E0EE53FD4F80815E
:10133000888387E894E060E00E948B2BE881F0E0EE
:10134000EE53FD4F80818883F801828193810B9752
:1013500018F18AE0A82EB12CA00EB11E750112C0A2
:10136000F701D1907F0187E894E06D2D0E948B2BCF
:10137000ED2DF0E0888190E0E827F927EE53FD4F4E
:10138000808188832E2D2A1930E0F8018281938193
:101390000A972817390720F3075F1E4F87E894E064
:1013A000F80160810E948B2BDF91CF911F910F91EB
:1013B000FF90EF90DF90BF90AF900895DF93CF93B1
:1013C000CDB7DEB7CA50D1400FB6F894DEBF0FBE1E
:1013D000CDBF2CE329836A832AE030E03C832B8352
:1013E000FC0184819581A681B7818D839E83AF8323
:1013F000B887CE0101960E94E208C65FDE4F0FB6A5
:10140000F894DEBF0FBECDBFCF91DF91089581EA82
:1014100096E06AE773E00E943A31882331F586E668
:1014200096E6A6E6B0E48093290690932A06A09358
:101430002B06B0932C0680E090E0A0E8BFE38093F9
:101440002D0690932E06A0932F06B093300688EEBB
:1014500093E0909332068093310681E880933306BF
:101460008DE8809334068DEF25C082E598EBAEE0E1
:10147000B0E48093290690932A06A0932B06B0939C
:101480002C0685E89BEEA1E5B0E480932D069093B1
:101490002E06A0932F06B093300680EA94E1909335
:1014A0003206809331068BEF8093330686E6809375
:1014B00034068AEF809335060895FF920F931F93A9
:1014C00001EA16E0C8016CE773E00E943A318093AC
:1014D0007006C8016EE773E00E943A31809371068E
:1014E000C80160E873E00E943A3180935006C80159
:1014F0006EE873E00E943A3180936806C8016AE89A
:1015000073E00E943A3180936606C80164E873E094
:101510000E943A3180937206C80166E873E00E9427
:101520003A3180937306C8016CE873E00E943A3147
:1015300080935806C80162E973E00E943A318093B3
:101540007406C80164E973E00E943A31809357063B
:10155000C80164EF73E00E943A31F82EC80165EFCC
:1015600073E00E943A31382F20E02F0D311D309367
:10157000760620937506C80166EF73E00E943A3143
:10158000F82EC80167EF73E00E943A31382F20E04F
:101590002F0D311D3093780620937706C80168EF30
:1015A00073E00E943A31F82EC80169EF73E00E949F
:1015B0003A31382F20E02F0D311D30937A062093D9
:1015C0007906C8016BEF73E00E943A3180934F06B1
:1015D0001F910F91FF900895BC0181EA96E00E944F
:1015E0003A3108956091D6047091D7048091D8045F
:1015F0009091D90420E030E040E152E40E94B536F9
:1016000020E030E044EB53E40E94E7340E941837B6
:101610000E944F359B012550304037FF03C09B018E
:10162000215E3F4FA8E3B6E0F901EE53FC4F808105
:101630008C932F5F3F4F2432310514F020E030E0CF
:10164000119686E0A334B80779F71C9208952F927B
:101650003F924F925F926F927F928F929F92AF9242
:10166000BF92CF92DF92EF92FF920F931F93DF937F
:10167000CF9300D000D000D0CDB7DEB7182F662EA4
:101680002091CC043091CD042A35310530F0C901C8
:101690008D549F4F89359105E8F437FF02C02D54D2
:1016A0003F4FC90137FF03C0909581959F4F8A3105
:1016B00091053CF0F4E48F2E912CE9ED2E2E312C87
:1016C0001DC00A975CF17BE3872E912C62ED262EDC
:1016D000312C20C02B35310514F0235B3040C9017B
:1016E00037FF03C0909581959F4F8A31910554F043
:1016F00056E5852E912C4CED242E312C37E0A32E6F
:10170000B12C15C00A9754F02DE4822E912C94ED43
:10171000292E312C88E0A82EB12C09C005E0802E9E
:10172000912CB8E32B2E312CA9E0AA2EB12C60917C
:10173000CE047091CF04882777FD8095982F0E9462
:10174000823527EA32E94BE25CEB0E94B5360E9413
:10175000893720E030E040EA50E40E94B53620E0CE
:1017600030E040E951E40E94B5360E94183720E08D
:1017700030E044E352E40E941A340E944F35712E47
:10178000FEEBCF2EFFEFDF2E9B01442737FD409568
:10179000542F29833A834B835C83E4EA4E2EE4E0A2
:1017A0005E2E4AEF5FEF240E351E6091CC047091DF
:1017B000CD04882777FD8095982F0E94823525E3F8
:1017C0003AEF4EE85CE30E94B5360E9489377B0110
:1017D0008C01B601882777FD8095982F0E9482356D
:1017E0009B01AC01C801B7010E94B5367B018C0199
:1017F00069817A818B819C810E9482359B01AC0139
:10180000C801B7010E941A340E944F359B01CB01D9
:1018100001978A35910508F071C062E170E00E947D
:10182000EF378B012F5F3F4FAEEEBFEF6A9FC001D6
:101830006B9F900D7A9F900D1124820F931F62E091
:1018400070E00E94EF376D837E83E62CE01A4E2D08
:101850004C5F84EA94E0672D0E94070500D000D019
:1018600000D0EDB7FEB73196ADB7BEB712965C9219
:101870004E92119720E031E0338322838D819E8147
:10188000880D991D958384830E94892A4DB75EB780
:101890004A5F5F4F0FB6F8945EBF0FBE4DBF8D819C
:1018A0009E818A159B0554F1043011053CF593E0A7
:1018B000E90EC201672D4E2D0E94070500D000D011
:1018C00000D0EDB7FEB73196ADB7BEB712965C92B9
:1018D0004E92119720E031E0338322834D815E8167
:1018E000420D531D558344830E94892A8DB79EB7AC
:1018F00006960FB6F8949EBF0FBE8DBFACE0B0E069
:10190000CA0EDB1E7394BEE4CB16D10409F04DCF92
:1019100026960FB6F894DEBF0FBECDBFCF91DF91F4
:101920001F910F91FF90EF90DF90CF90BF90AF90FD
:101930009F908F907F906F905F904F903F902F90EF
:101940000895823010F422E002C0282F220F30E0E8
:101950008DB79EB708970FB6F8949EBF0FBE8DBF88
:10196000EDB7FEB7319684EA94E0ADB7BEB71296F4
:101970009C938E93119783E091E093838283225707
:101980003F4F358324832F5F3F4F378326830E9449
:10199000892A8DB79EB708960FB6F8949EBF0FBEE2
:1019A0008DBF0895CF93DF93AC01E091DE04F091F9
:1019B000DF042091360630913706C9018C599F4FBC
:1019C0008E179F071CF4EA01219709C02456304066
:1019D000E217F30714F0EA0102C0EA012196842F0E
:1019E00090E0C817D90729F081EA96E04C2F0E94B1
:1019F0004131CE01DF91CF9108950F931F9301EAFA
:101A000016E0C80163EF73E041E00E944131C80174
:101A100064EF73E043E10E944131C80165EF73E078
:101A200046E00E944131C80166EF73E040E10E9448
:101A30004131C80167EF73E047E20E944131C801BC
:101A400068EF73E048E80E944131C80169EF73E034
:101A500043E10E9441311F910F910895CF92DF928F
:101A6000EF92FF920F931F937C01D62EC72E04EAAC
:101A700014E0C8016E2D4D2D0E947004C8010E9413
:101A8000480500D000D0EDB7FEB71283018383E391
:101A900091E0948383830E94782AEDB7FEB7128386
:101AA000018383E291E0948383830E94782AEDB7D7
:101AB000FEB71283018383E191E0948383830E94C4
:101AC000782AEDB7FEB71283018383E091E0948317
:101AD00083830E94782AEDB7FEB71283018384EFD7
:101AE00090E0948383830E94782A0F900F900F9048
:101AF0000F90C8010E942C05C70101966D2D7C2D09
:101B00000E94270B1F910F91FF90EF90DF90CF90D5
:101B10000895CF92DF92EF92FF920F931F93CF938E
:101B2000DF93182F062F0E94223228EE33E040E088
:101B300050E00E94023869017A01C4EAD4E0CE0183
:101B4000612F402F0E947004CE010E9448058091B1
:101B5000FE049091FF04892B09F453C00091000505
:101B6000109101058DB79EB744970FB6F8949EBFAC
:101B70000FBE8DBFEDB7FEB73196ADB7BEB71296AB
:101B8000DC93CE93119788E091E09383828383EB7B
:101B900090E095838483C6016CE370E00E94EF3788
:101BA000CB016CE370E00E94EF37978386832AE3D2
:101BB00030E031872087C6016CE370E00E94EF3788
:101BC0009387828785E690E095878487C8016CE3D8
:101BD00070E00E94DB37CB016CE370E00E94EF37CE
:101BE00097878687318B208BC8016CE370E00E9459
:101BF000DB37938B828B0E94892A8DB79EB74496E0
:101C000033C0ADB7BEB71C970FB6F894BEBF0FBEBA
:101C1000ADBFEDB7FEB731961296DC93CE93119718
:101C200080E291E09383828383EB90E095838483C9
:101C3000C6016CE370E00E94EF37CB016CE370E00B
:101C40000E94EF37978386838AE390E091878087AD
:101C5000C6016CE370E00E94EF37938782870E9491
:101C6000892A8DB79EB70C960FB6F8949EBF0FBE0B
:101C70008DBF84EA94E00E942C05DF91CF911F91E3
:101C80000F91FF90EF90DF90CF900895EF92FF9229
:101C90000F931F93282F462FA4EAEA2EA4E0FA2ED2
:101CA000C701622F0E947004C7010E9448058DB7CA
:101CB0009EB70A970FB6F8949EBF0FBE8DBF0DB7A3
:101CC0001EB70F5F1F4FEDB7FEB7F282E1828CE2C5
:101CD00091E0F8019383828360910205709103057E
:101CE000809104059091050520912D0630912E06D6
:101CF00040912F06509130060E94B536F80164835A
:101D000075838683978380EB90E0918780870E941C
:101D1000892A8DB79EB70A960FB6F8949EBF0FBE5C
:101D20008DBFC7010E942C051F910F91FF90EF906E
:101D300008958F929F92AF92BF92CF92DF92EF92CF
:101D4000FF920F931F93E82EF62E04EA14E0C801C9
:101D50006E2D4F2D0E947004C8010E9448058DB75A
:101D60009EB70C970FB6F8949EBF0FBE8DBFEDB710
:101D7000FEB73196ADB7BEB712961C930E9311976E
:101D800094E3892E91E0992E938282828DEEA82E83
:101D9000B12CB582A48280910B0590910C05A09185
:101DA0000D05B0910E0586839783A087B187B3EFA9
:101DB000CB2ED12CD386C2860E94892A8DB79EB79E
:101DC0000C960FB6F8949EBF0FBE8DBFC8010E943F
:101DD0002C05F394C8016E2D4F2D0E947004C8018C
:101DE0000E944805ADB7BEB71C970FB6F894BEBFAA
:101DF0000FBEADBFEDB7FEB7319612961C930E9392
:101E0000119793828282B582A48280910F0590916E
:101E10001005A0911105B091120586839783A087C4
:101E2000B187D386C2860E94892A8DB79EB70C9649
:101E30000FB6F8949EBF0FBE8DBFC8010E942C053F
:101E4000F394C8016E2D4F2D0E947004C8010E94AA
:101E50004805ADB7BEB71C970FB6F894BEBF0FBE0E
:101E6000ADBFEDB7FEB7319612961C930E93119746
:101E700093828282B582A482809113059091140589
:101E8000A0911505B091160586839783A087B18729
:101E9000D386C2860E94892A8DB79EB70C960FB64C
:101EA000F8949EBF0FBE8DBFC8010E942C051F91E4
:101EB0000F91FF90EF90DF90CF90BF90AF909F90E9
:101EC0008F9008950F931F93282F462F04EA14E054
:101ED000C801622F0E947004C8010E9448058DB796
:101EE0009EB70A970FB6F8949EBF0FBE8DBFEDB791
:101EF000FEB73196ADB7BEB712961C930E931197ED
:101F00008EE391E09383828389EB90E095838483D1
:101F10008091FE049091FF049783868382E890E08D
:101F2000918780870E94892A8DB79EB70A960FB63F
:101F3000F8949EBF0FBE8DBFC8010E942C051F9153
:101F40000F910895EF92FF920F931F93282F462F22
:101F500034EAE32E34E0F32EC701622F0E947004AE
:101F6000C7010E9448058DB79EB70C970FB6F8942D
:101F70009EBF0FBE8DBF0DB71EB70F5F1F4FEDB7D2
:101F8000FEB7F282E18286E491E0F80193838283D6
:101F900084EE90E0958384836091FC047091FD044D
:101FA000882777FD8095982F0E9482352AE037EDAB
:101FB00043E25CE30E94B536F8016683778380874D
:101FC00091878FE890E0938782870E94892A8DB756
:101FD0009EB70C960FB6F8949EBF0FBE8DBFC7017B
:101FE0000E942C051F910F91FF90EF9008950F9381
:101FF0001F93282F462F04EA14E0C801622F0E9485
:102000007004C8010E9448058DB79EB70C970FB6A3
:10201000F8949EBF0FBE8DBFEDB7FEB73196ADB73A
:10202000BEB712961C930E93119786E491E09383AA
:10203000828382EE90E0958384838091F80490916E
:10204000F904A091FA04B091FB0486839783A087DA
:10205000B1878EE890E0938782870E94892A8DB7A6
:102060009EB70C960FB6F8949EBF0FBE8DBFC801E9
:102070000E942C051F910F9108950F931F93282FF5
:10208000462F84EA94E0622F0E94700484EA94E070
:102090000E9448058091DB04882319F420E531E093
:1020A00057C0813019F424E531E052C0823019F470
:1020B00028E531E04DC0833019F42CE531E048C00B
:1020C000843019F420E631E043C0853019F424E669
:1020D00031E03EC0863019F428E631E039C087305F
:1020E00019F42CE631E034C0883019F420E731E0EF
:1020F0002FC0893019F424E731E02AC08A3019F45E
:1021000028E731E025C08B3019F42CE731E020C0FE
:102110008C3019F420E831E01BC08D3019F424E82C
:1021200031E016C08E3019F428E831E011C08F304C
:1021300019F42CE831E00CC0803119F420E931E0C9
:1021400007C0813119F024E931E002C025E931E00E
:102150008DB79EB708970FB6F8949EBF0FBE8DBF80
:10216000EDB7FEB7319604EA14E0ADB7BEB71296EC
:102170001C930E93119789E991E09383828380EEFB
:1021800090E095838483378326830E94892A8DB7C4
:102190009EB708960FB6F8949EBF0FBE8DBFC801BC
:1021A0000E942C051F910F9108950F931F93282FC4
:1021B000462F04EA14E0C801622F0E947004C8018F
:1021C0000E9448058DB79EB70A970FB6F8949EBF38
:1021D0000FBE8DBFEDB7FEB73196ADB7BEB7129645
:1021E0001C930E9311978EE991E09383828387E885
:1021F00090E0958384838091DC049091DD04978343
:10220000868385E290E0918780870E94892A8DB736
:102210009EB70A960FB6F8949EBF0FBE8DBFC80139
:102220000E942C051F910F9108950F931F93282F43
:10223000462F04EA14E0C801622F0E947004C8010E
:102240000E9448058DB79EB70A970FB6F8949EBFB7
:102250000FBE8DBFEDB7FEB73196ADB7BEB71296C4
:102260001C930E93119788EA91E093838283809167
:10227000CE049091CF049583848380EB90E0978384
:10228000868381EB90E0918780870E94892A8DB7B1
:102290009EB70A960FB6F8949EBF0FBE8DBFC801B9
:1022A0000E942C051F910F9108950F931F93282FC3
:1022B000462F04EA14E0C801622F0E947004C8018E
:1022C0000E9448058DB79EB70A970FB6F8949EBF37
:1022D0000FBE8DBFEDB7FEB73196ADB7BEB7129644
:1022E0001C930E93119788EA91E0938382838091E7
:1022F000CC049091CD049583848380EB90E0978308
:10230000868382EB90E0918780870E94892A8DB72F
:102310009EB70A960FB6F8949EBF0FBE8DBFC80138
:102320000E942C051F910F9108950F931F93282F42
:10233000462F04EA14E0C801622F0E947004C8010D
:102340000E9448058DB79EB70A970FB6F8949EBFB6
:102350000FBE8DBFEDB7FEB73196ADB7BEB71296C3
:102360001C930E93119780EB91E09383828381EE0F
:1023700090E0958384838091AB029091AC02978327
:10238000868385E290E0918780870E94892A8DB7B5
:102390009EB70A960FB6F8949EBF0FBE8DBFC801B8
:1023A0000E942C051F910F9108950F931F93282FC2
:1023B000462F04EA14E0C801622F0E947004C8018D
:1023C0000E9448058DB79EB70C970FB6F8949EBF34
:1023D0000FBE8DBFEDB7FEB73196ADB7BEB7129643
:1023E0001C930E93119788EB91E09383828382EC88
:1023F00091E09583848380ED90E09783868388E3E2
:1024000096E09187808781ED90E0938782870E9494
:10241000892A8DB79EB70C960FB6F8949EBF0FBE53
:102420008DBFC8010E942C051F910F9108950F9335
:102430001F93282F462F04EA14E0C801622F0E9440
:102440007004C8010E9448058DB79EB70A970FB661
:10245000F8949EBF0FBE8DBFEDB7FEB73196ADB7F6
:10246000BEB712961C930E93119780ED91E0938363
:1024700082838091D6049091D704A091D804B09122
:10248000D90484839583A683B78380EB90E09187FA
:1024900080870E94892A8DB79EB70A960FB6F89456
:1024A0009EBF0FBE8DBFC8010E942C051F910F91CA
:1024B00008950F931F93282F462F04EA14E0C801B4
:1024C000622F0E947004C8010E9448058DB79EB714
:1024D0000C970FB6F8949EBF0FBE8DBFEDB7FEB739
:1024E0003196ADB7BEB712961C930E93119788ED37
:1024F00091E09383828386E190E095838483809149
:10250000F0049091F104A091F204B091F304868359
:102510009783A087B18788E890E0938782870E949D
:10252000892A8DB79EB70C960FB6F8949EBF0FBE42
:102530008DBFC8010E942C051F910F910895CF9265
:10254000DF92EF92FF920F931F93CF93DF93282F89
:10255000462FC4EAD4E0CE01622F0E947004CE015F
:102560000E94480560914406709145068091460698
:102570009091470620912D0630912E0640912F060E
:10258000509130060E94B5366B017C0120E030E0AE
:102590004AE754E40E94AA361816D4F58DB79EB7C0
:1025A0000C970FB6F8949EBF0FBE8DBF0DB71EB728
:1025B0000F5F1F4FADB7BEB71296DC93CE93119746
:1025C00086E491E0F801938382838EEF90E0958317
:1025D00084836091310670913206882777FD80955B
:1025E000982F0E9482359B01AC01C701B6010E9461
:1025F000E734D80116966D937D938D939C9319972C
:10260000809135061A968C931A971B961C9221C0BE
:102610008DB79EB70C970FB6F8949EBF0FBE8DBFB7
:10262000EDB7FEB73196ADB7BEB71296DC93CE9339
:10263000119782EE91E0938382838EEF90E09583F1
:102640008483C682D782E086F186809134068287B1
:1026500013860E94892AEDB7FEB73C960FB6F89410
:10266000FEBF0FBEEDBF84EA94E00E942C05DF910F
:10267000CF911F910F91FF90EF90DF90CF90089531
:10268000EF92FF920F931F93282F462F54EAE52EC7
:1026900054E0F52EC701622F0E947004C7010E940A
:1026A00048058DB79EB70C970FB6F8949EBF0FBE26
:1026B0008DBF0DB71EB70F5F1F4FEDB7FEB7F2828C
:1026C000E18288ED91E0F8019383828389EE90E0C6
:1026D000958384836091EC047091ED048091EE0405
:1026E0009091EF042091290630912A0640912B0603
:1026F00050912C060E94B536F80166837783808757
:10270000918780913306828713860E94892A8DB72C
:102710009EB70C960FB6F8949EBF0FBE8DBFC70133
:102720000E942C051F910F91FF90EF900895EF925A
:10273000FF920F931F93282F462F64EAE62E64E042
:10274000F62EC701622F0E947004C7010E9448053F
:102750008DB79EB70C970FB6F8949EBF0FBE8DBF76
:102760000DB71EB70F5F1F4FEDB7FEB7F282E182C4
:1027700088ED91E0F8019383828388EE90E0958361
:1027800084836091F4047091F5048091F604909133
:10279000F7042091290630912A0640912B0650918A
:1027A0002C060E94B536F80166837783808791876F
:1027B00080913306828713860E94892A8DB79EB73F
:1027C0000C960FB6F8949EBF0FBE8DBFC7010E9436
:1027D0002C051F910F91FF90EF900895EF92FF92BB
:1027E0000F931F93282F462F74EAE72E74E0F72EDD
:1027F000C701622F0E947004C7010E9448058DB76F
:102800009EB70C970FB6F8949EBF0FBE8DBF0DB745
:102810001EB70F5F1F4FEDB7FEB7F282E18282EE67
:1028200091E0F8019383828386EE90E09583848320
:102830006091E8047091E9048091EA049091EB04BE
:1028400020912D0630912E0640912F065091300692
:102850000E94B536F80166837783808791878091DF
:102860003406828713860E94892A8DB79EB70C96FC
:102870000FB6F8949EBF0FBE8DBFC7010E942C05F6
:102880001F910F91FF90EF900895EF92FF920F9399
:102890001F93282F462FE4EAEE2EE4E0FE2EC70118
:1028A000622F0E947004C7010E9448058DB79EB731
:1028B0000C970FB6F8949EBF0FBE8DBF0DB71EB715
:1028C0000F5F1F4FEDB7FEB7F282E18282EE91E01B
:1028D000F8019383828387EE90E0958384836091EF
:1028E000060570910705882777FD8095982F0E942F
:1028F000823520912D0630912E0640912F06509161
:1029000030060E94B536F801668377838087918709
:1029100080913406828713860E94892A8DB79EB7DC
:102920000C960FB6F8949EBF0FBE8DBFC7010E94D4
:102930002C051F910F91FF90EF9008950F931F9317
:10294000282F462F04EA14E0C801622F0E94700469
:10295000C8010E944805809148060E94A10CC80148
:102960000E942C051F910F910895EF92FF920F93F3
:102970001F93282F462FF4EAEF2EF4E0FF2EC70115
:10298000622F0E947004C7010E9448058DB79EB750
:102990000C970FB6F8949EBF0FBE8DBF0DB71EB734
:1029A0000F5F1F4FEDB7FEB7F282E18282EE91E03A
:1029B000F801938382838FE190E095838483609113
:1029C000490670914A0680914B0690914C060E94F0
:1029D000823520912D0630912E0640912F06509180
:1029E00030060E94B536F801668377838087918729
:1029F00080913406828713860E94892A8DB79EB7FC
:102A00000C960FB6F8949EBF0FBE8DBFC7010E94F3
:102A10002C051F910F91FF90EF9008950F931F9336
:102A2000282F462F04EA14E0C801622F0E94700488
:102A3000C8010E9448058DB79EB740970FB6F8941D
:102A40009EBF0FBE8DBFEDB7FEB73196ADB7BEB717
:102A500012961C930E9311978CEE91E093838283D0
:102A600083E890E0958384838091D2049091D3048D
:102A7000A091D404B091D50486839783A087B187B1
:102A800084E890E0938782878091E2049091E30448
:102A9000A091E404B091E50484879587A687B78761
:102AA0000E94892A8DB79EB740960FB6F8949EBFB4
:102AB0000FBE8DBFC8010E942C051F910F91089574
:102AC0000F931F93282F462F84EA94E0622F0E94D1
:102AD000700484EA94E00E9448058091E704282F5E
:102AE00030E0823030F4A4E0220F331FAA95E1F7E2
:102AF00002C02150304000D000D000D0EDB7FEB76A
:102B0000319604EA14E0ADB7BEB712961C930E934B
:102B1000119780E091E093838283358324830E9420
:102B2000892A8DB79EB706960FB6F8949EBF0FBE42
:102B30008DBFC8010E942C051F910F9108950F931E
:102B40001F93282F462F04EA14E0C801622F0E9429
:102B50007004C8010E9448058DB79EB708970FB64C
:102B6000F8949EBF0FBE8DBFEDB7FEB73196ADB7DF
:102B7000BEB712961C930E9311978EEF91E093833C
:102B800082838FE090E0958384838091E60486833E
:102B900017820E94892A8DB79EB708960FB6F894BF
:102BA0009EBF0FBE8DBFC8010E942C051F910F91C3
:102BB00008950F931F9304EA14E0C80163E045E011
:102BC0000E947004C8010E94480500D000D0EDB7F3
:102BD000FEB7128301838FE591E0948383830E9483
:102BE000782AEDB7FEB71283018386E591E09483DE
:102BF00083830E94782AEDB7FEB71283018380E5B4
:102C000091E0948383830E94782AEDB7FEB7128304
:102C1000018389E491E0948383830E94782AEDB74D
:102C2000FEB71283018383E491E0948383830E943F
:102C3000782A0F900F900F900F90C8010E942C05DA
:102C40001F910F9108950F931F93282F462F04EA89
:102C500014E0C801622F0E947004C8010E94480558
:102C600000D000D0EDB7FEB71283018386E791E074
:102C7000948383830E94782A0F900F900F900F9077
:102C8000C8010E942C051F910F910895EF92FF92A9
:102C90000F931F93CF93DF930E942232209152060D
:102CA0003091530640915406509155062617370728
:102CB0004807590708F08AC10E9422326C507E4FA3
:102CC0008F4F9F4F60935206709353068093540624
:102CD0009093550604EA14E0C8010E949505C801C6
:102CE00065E043E00E947004C8010E94480500D0DE
:102CF00000D0EDB7FEB71283018386ED91E0948397
:102D000083830E94782A0F900F900F900F908091EC
:102D1000360690913706892B31F080914D069091BF
:102D20004E06892B81F48091DE049091DF0490930C
:102D30003706809336068091E0049091E1049093E9
:102D40004E0680934D062091E0043091E1044091BD
:102D50004D0650914E06C9018456904048175907B8
:102D600024F4809151068F5F08C02C593F4F2417DF
:102D700035072CF480915106815080935106809143
:102D80005106181614F081E003C084301CF083E073
:102D90008093510680915106823009F462C08330DD
:102DA00009F4BEC0813009F00DC100D000D0C4EAE2
:102DB000D4E0EDB7FEB7D283C1838DEC91E094836C
:102DC00083830E94782A809127060F900F900F909E
:102DD0000F9080FF22C000D000D0EDB7FEB7D283A5
:102DE000C18385EC91E0948383830E94782A80914B
:102DF000360690913706845690400F900F900F90B2
:102E00000F902091DE043091DF04281739070CF071
:102E1000D9C0809127068E7F21C000D000D0EDB7A9
:102E2000FEB7D283C1838DEB91E0948383830E94AC
:102E3000782A80913606909137068C599F4F0F90D3
:102E40000F900F900F902091DE043091DF048217D5
:102E500093070CF0B7C08091270681608093270606
:102E6000B1C000D000D0C4EAD4E0EDB7FEB7D28341
:102E7000C18383EB91E0948383830E94782A0F902F
:102E80000F900F900F9080914F06882301F100D092
:102E900000D0EDB7FEB7D283C18389EA91E0948375
:102EA00083830E94782A8091360690913706845653
:102EB00090400F900F900F900F902091DE04309172
:102EC000DF04281739071CF510924F0620C000D0E8
:102ED00000D0EDB7FEB7D283C1838CE991E0948333
:102EE00083830E94782A80913606909137068C5908
:102EF0009F4F0F900F900F900F902091DE04309114
:102F0000DF04821793071CF481E080934F0681EA67
:102F100096E06BEF73E040914F060E94413152C042
:102F200000D000D0B4EAEB2EB4E0FB2EEDB7FEB734
:102F3000F282E1828BE891E0948383830E94782A75
:102F40008DB79EB708970FB6F8949EBF0FBE8DBF82
:102F50000DB71EB70F5F1F4FEDB7FEB7F282E182CC
:102F600084E092E0F801938382836091500670E0E0
:102F700080E090E00E94803520E030E040E251E4C3
:102F80000E94E734F801648375838683978386E71C
:102F900090E09187808780E290E0938782870E940B
:102FA000892A8DB79EB70C960FB6F8949EBF0FBEB8
:102FB0008DBF8091500690E060E873E00E94D20CD3
:102FC0008093500684EA94E00E942C05DF91CF9113
:102FD0001F910F91FF90EF900895BF92CF92DF92D3
:102FE000EF92FF920F931F93CF93DF93E82ED62E8D
:102FF0000E94223220915F06309160064091610666
:1030000050916206261737074807590708F024C170
:10301000809163068823C9F08093AD021092630605
:103020008CE092E090936506809364060E942232C1
:103030006C507E4F8F4F9F4F60935F06709360067A
:103040008093610690936206C2C08091AD02A82F62
:10305000B0E07091DA044091640650916506F090FA
:10306000C7041091E7040091560660911805E0919D
:10307000AB02F091AC0280915706C82FD0E0B0901F
:103080005806909117059D012F5F3F4F273031055E
:103090001CF021E030E019C02330310531F124303B
:1030A000310544F42130310581F02230310509F039
:1030B00057C012C02530310591F125303105ECF0B3
:1030C0002630310509F04CC037C0723008F048C0D6
:1030D00049E152E081E049C083E0C82EFC1409F4C4
:1030E0003FC046E252E082E040C01230C8F5002303
:1030F000B9F143E352E083E038C0623088F16330D5
:1031000039F0643041F0623041F440E452E005C0EF
:103110004DE452E002C04AE552E084E026C0EC17DC
:10312000FD07F4F48FEFED39F807D1F0BB20C1F4BF
:1031300047E652E085E019C0723090F4923080F09A
:10314000933039F0943041F0923051F444E752E03A
:1031500005C040E852E002C04DE852E086E005C0FC
:103160002A173B0709F090CF60C050936506409343
:1031700064068093630681E0809359060E942232A0
:1031800068517C4F8F4F9F4F60935F06709360062E
:1031900080936106909362060E9422326056704FBF
:1031A0008F4F9F4F60935B0670935C0680935D0624
:1031B00090935E0680915A06882321F084EA94E079
:1031C0000E94950510925A0602C01092590604EA10
:1031D00014E0C8016E2D4D2D0E947004C8010E949C
:1031E000480500D000D000D0EDB7FEB73196ADB79E
:1031F000BEB712961C930E9311978AE992E09383BF
:1032000082838091640690916506958384830E94F1
:10321000892A8DB79EB706960FB6F8949EBF0FBE4B
:103220008DBFC8010E942C0517C0509365064093BE
:103230006406109263060E94223220915B06309150
:103240005C0640915D0650915E06261737074807D9
:10325000590708F4BACFBBCFDF91CF911F910F91DF
:10326000FF90EF90DF90CF90BF900895EF92FF9284
:103270000F931F9380916606843009F056C0909199
:10328000DB04943008F027C180916F068917A1F103
:1032900090936F060E94223260936B0670936C06C7
:1032A00080936D0690936E0690916F068091AE02AA
:1032B000981711F580915A06813091F0813018F0FD
:1032C0008230B1F413C011E010935A060E942232EA
:1032D000615375478040904030F41093670608C0F2
:1032E00082E080935A061092670602C010925A0636
:1032F00084EA94E00E9495050E94223220916B0698
:1033000030916C0640916D0650916E06621B730BF6
:10331000840B950B615D77408040904008F4DBC0E2
:103320008091DB048093AE02D6C0853029F4809171
:10333000A3029091A40214C0863029F48091A502C2
:103340009091A6020DC0873029F48091A702909138
:10335000A80206C0883041F48091A9029091AA0287
:1033600090936A06809369068091680620916906A9
:1033700030916A06882309F04AC0C90189509740F4
:103380008F5A9440C8F40E9422326153754780409E
:10339000904020F481E0809367060CC0809167061E
:1033A000882341F480915906882321F484EA94E02B
:1033B0000E94950582E028C044E0203B340768F471
:1033C00080915A06882349F01092670684EA94E0B7
:1033D0000E94950510925A067EC0205B3440295504
:1033E000324008F078C080915A06813009F473C0E9
:1033F00080915906882309F06EC01092670684EA0E
:1034000094E00E94950581E080935A0664C0215B98
:10341000344008F460C00E942232615375478040F6
:10342000904008F041C0809167068823E9F5E0905C
:103430006B06F0906C0600916D0610916E0688EE9A
:1034400093E0A0E0B0E0E80EF91E0A1F1B1F0E94E7
:103450002232E616F70608071907E8F581E080939F
:10346000670617C01092670684EA94E00E949505EB
:1034700080915A06823019F410925A0603C08F5F69
:1034800080935A0680915A06823018F082E0809329
:103490005A060E94223260936B0670936C068093EA
:1034A0006D0690936E0617C0E0906B06F0906C0668
:1034B00000916D0610916E0688EE93E0A0E0B0E0FA
:1034C000E80EF91E0A1F1B1F0E942232E616F7069D
:1034D0000807190738F21F910F91FF90EF90089598
:1034E00080916606843010F00E943619809167063C
:1034F000882319F00E94461608958091070480FFE2
:1035000008C060916D0480916B0490E070E00E94AF
:10351000ED1780915A06823008F012C2A82FB0E051
:10352000FD01EF5FFB4F808185FF0BC0FD01E35E76
:10353000FB4F6081A55EBB4F8C9190E070E00E94D4
:103540009F1580915A06A82FB0E0FD01EF5FFB4F59
:10355000808186FF0BC0FD01EF5DFB4F6081A15EA6
:10356000BB4F8C9190E070E00E94601580915606F0
:10357000882309F43FC080915A06A82FB0E0FD01CE
:10358000EF5FFB4F808187FF0BC0FD01EB5DFB4FC1
:103590006081AD5DBB4F8C9190E070E00E940E1594
:1035A00080915A06A82FB0E0FD01ED5FFB4F8081AE
:1035B00084FF0BC0FD01E35CFB4F6081A55CBB4F4A
:1035C0008C9190E070E00E94B51480915A06A82F6B
:1035D000B0E0FD01ED5FFB4F808183FF0BC0FD017B
:1035E000E75CFB4F6081A95CBB4F8C9190E070E081
:1035F0000E949E1480915A06A82FB0E0FD01EB5F57
:10360000FB4F808187FF0BC0FD01EB5AFB4F6081B0
:10361000AD5ABB4F8C9190E070E00E9445148091B0
:103620005A06A82FB0E0FD01E95FFB4F808183FFC0
:103630000BC0FD01EB58FB4F6081AD58BB4F8C9127
:1036400090E070E00E94591280915A06A82FB0E0D5
:10365000FD01EB5FFB4F808181FF0BC0FD01E35A51
:10366000FB4F6081A55ABB4F8C9190E070E00E94A7
:10367000971380915606882309F444C08091E7048B
:10368000823008F43FC080915A06A82FB0E0FD01B7
:10369000E75FFB4F808182FF0BC0FD01EF57FB4FBF
:1036A0006081A158BB4F8C9190E070E00E949F1206
:1036B00080915A06A82FB0E0FD01EB5FFB4F80819F
:1036C00082FF0BC0FD01EF5AFB4F6081A15BBB4F36
:1036D0008C9190E070E00E94EE1380915A06A82F22
:1036E000B0E0FD01EB5FFB4F808183FF0BC0FD016C
:1036F000E75AFB4F6081A95ABB4F8C9190E070E074
:103700000E94401380915A06A82FB0E0FD01ED5FA2
:10371000FB4F808181FF0BC0FD01EF5CFB4F60819F
:10372000A15DBB4F8C9190E070E00E9417128091D8
:103730005A06A82FB0E0FD01ED5FFB4F808180FFAE
:103740000BC0FD01E35DFB4F6081A55DBB4F8C911C
:1037500090E070E00E94D51180915A06A82FB0E049
:10376000FD01E95FFB4F808186FF0BC0FD01E3583F
:10377000FB4F6081A558BB4F8C9190E070E00E9498
:10378000951180915A06A82FB0E0FD01EF5FFB4F25
:10379000808182FF0BC0FD01EB5EFB4F6081AD5E5F
:1037A000BB4F8C9190E070E00E94551180915A06B9
:1037B000A82FB0E0FD01EF5FFB4F808181FF0BC0C0
:1037C000FD01EF5EFB4F6081A15FBB4F8C9190E0EC
:1037D00070E00E94151180915A06A82FB0E0FD01FB
:1037E000EB5FFB4F808184FF0BC0FD01EF59FB4F66
:1037F0006081A15ABB4F8C9190E070E00E94D5107F
:1038000080915A06A82FB0E0FD01EB5FFB4F80814D
:1038100085FF0BC0FD01EB59FB4F6081AD59BB4FDC
:103820008C9190E070E00E943D1080915A06A82F84
:10383000B0E0FD01EF5FFB4F808183FF0BC0FD0116
:10384000E75EFB4F6081A95EBB4F8C9190E070E01A
:103850000E94F70F80915A06A82FB0E0FD01EB5FA0
:10386000FB4F808180FF0BC0FD01E35BFB4F60815C
:10387000A55BBB4F8C9190E070E00E94A20F8091FD
:103880005A06A82FB0E0FD01EF5FFB4F808184FF57
:103890000BC0FD01E75DFB4F6081A95DBB4F8C91C3
:1038A00090E070E00E94620F80915A06A82FB0E06D
:1038B000FD01E75FFB4F808181FF18C080914F06BB
:1038C000FD01ED57FB4F813049F4AB57BB4F6C9175
:1038D000808190E070E00E94460E08C0AB57BB4F5D
:1038E0006C91808190E070E00E94990E80915A0660
:1038F000A82FB0E0FD01ED5FFB4F808187FF0BC07B
:10390000FD01E75BFB4F6081A95BBB4F8C9190E0B1
:1039100070E00E94890D80915A06A82FB0E0FD0149
:10392000EB5FFB4F808186FF0BC0FD01E759FB4F2A
:103930006081A959BB4F8C9190E070E00E942E0DE0
:10394000089584EA94E00E9495050E94D9150E948A
:10395000070A0895CF93DF93EC0184EA94E00E9474
:103960006C04C817D9073CF084EA94E00E94610413
:10397000892B09F42397CE01DF91CF910895EF921F
:10398000FF920F931F93CF93DF9300915A0610E09D
:103990008AEF90E0089F7001099FF00C189FF00CCF
:1039A0001124C7010E94EC0AF801EF5FFB4F882346
:1039B00019F08081816002C080818E7F8083809138
:1039C0005A06C82FD0E0C70102960E94EC0AC55FD4
:1039D000DB4F888380915A06C82FD0E0C701049638
:1039E0000E94EC0A90E00E94AA1CC35FDB4F888310
:1039F00000915A0610E0C70188569F4F0E94EC0ABA
:103A0000F801EF5FFB4F882319F08081806102C0CD
:103A100080818F7E808380915A06C82FD0E0C701B5
:103A200086569F4F0E94EC0AC95DDB4F88838091C8
:103A30005A06C82FD0E0C70184569F4F0E94EC0A57
:103A400090E00E94AA1CC75DDB4F888300915A0654
:103A500010E0C70106960E94EC0AF801EF5FFB4FE9
:103A6000882319F08081826002C080818D7F8083ED
:103A700080915A06C82FD0E0C70108960E94EC0A30
:103A8000C15FDB4F888380915A06C82FD0E0C70101
:103A90000A960E94EC0A90E00E94AA1CCF5EDB4FBF
:103AA000888300915A0610E0C7010C960E94EC0A28
:103AB000F801EF5FFB4F882319F08081846002C01A
:103AC00080818B7F808380915A06C82FD0E0C70108
:103AD0000E960E94EC0ACD5EDB4F888380915A06D9
:103AE000C82FD0E0C70140960E94EC0A90E00E94E7
:103AF000AA1CCB5EDB4F888300915A0610E0C701F9
:103B000042960E94EC0AF801EF5FFB4F882319F000
:103B10008081886002C08081877F808380915A067F
:103B2000C82FD0E0C70144960E94EC0AC95EDB4F63
:103B3000888380915A06C82FD0E0C70146960E941C
:103B4000EC0A90E00E94AA1CC75EDB4F88830091BC
:103B50005A0610E0C7014E960E94EC0AF801EF5F8A
:103B6000FB4F882319F08081806202C080818F7DA5
:103B7000808380915A06C82FD0E0C70180960E94AA
:103B8000EC0AC55EDB4F888380915A06C82FD0E0CF
:103B9000C70182960E94EC0A90E00E94AA1CC35EB4
:103BA000DB4F888300915A0610E0C70184960E947B
:103BB000EC0AF801EF5FFB4F882319F080818064E5
:103BC00002C080818F7B808380915A06C82FD0E00D
:103BD000C70186960E94EC0AC15EDB4F8883809104
:103BE0005A06C82FD0E0C70188960E94EC0A90E0E0
:103BF0000E94AA1CCF5DDB4F888300915A0610E01B
:103C0000C7018A960E94EC0AF801EF5FFB4F8823F8
:103C100019F08081806802C080818F7780838091D5
:103C20005A06C82FD0E0C7018C960E94EC0ACD5DE1
:103C3000DB4F888380915A06C82FD0E0C7018E964B
:103C40000E94EC0A90E00E94AA1CCB5DDB4F8883A7
:103C500000915A0610E0C701C0960E94EC0AF801D4
:103C6000ED5FFB4F882319F08081816002C0808165
:103C70008E7F808380915A06C82FD0E0C701C296FC
:103C80000E94EC0AC55DDB4F888380915A06C82FDD
:103C9000D0E0C701C4960E94EC0A90E00E94AA1CE2
:103CA000C35DDB4F888300915A0610E0C701C696BA
:103CB0000E94EC0AF801ED5FFB4F882319F0808128
:103CC000826002C080818D7F808380915A06C82FD8
:103CD000D0E0C701C8960E94EC0AC15DDB4F888323
:103CE00080915A06C82FD0E0C701CA960E94EC0AFC
:103CF00090E00E94AA1CCF5CDB4F888300915A069B
:103D000010E0C701CC960E94EC0AF801ED5FFB4F72
:103D1000882319F08081846002C080818B7F80833A
:103D200080915A06C82FD0E0C701CE960E94EC0AB7
:103D3000CD5CDB4F888380915A06C82FD0E0C70145
:103D4000805C9F4F0E94EC0A90E00E94AA1CCB5C12
:103D5000DB4F888300915A0610E0C701885B9F4FB4
:103D60000E94EC0AF801ED5FFB4F882319F0808177
:103D7000806102C080818F7E808380915A06C82F27
:103D8000D0E0C701865B9F4F0E94EC0AC55CDB4F09
:103D9000888380915A06C82FD0E0C701845B9F4F6B
:103DA0000E94EC0A90E00E94AA1CC35CDB4F88834F
:103DB00000915A0610E0C7018E5B9F4F0E94EC0AEB
:103DC000F801ED5FFB4F882319F08081886002C005
:103DD0008081877F808380915A06C82FD0E0C701F9
:103DE0008C5B9F4F0E94EC0AC95CDB4F88838091FB
:103DF0005A06C82FD0E0C7018A5B9F4F0E94EC0A89
:103E000090E00E94AA1CC75CDB4F888300915A0691
:103E100010E0C701805B9F4F0E94EC0AF801ED5F44
:103E2000FB4F882319F08081806202C080818F7DE2
:103E3000808380915A06C82FD0E0C7018E5A9F4FC9
:103E40000E94EC0AC15CDB4F888380915A06C82F20
:103E5000D0E0C7018C5A9F4F0E94EC0A90E00E946C
:103E6000AA1CCF5BDB4F888300915A0610E0C70184
:103E70008A5A9F4F0E94EC0AF801ED5FFB4F88239E
:103E800019F08081806402C080818F7B8083809163
:103E90005A06C82FD0E0C701885A9F4F0E94EC0AEB
:103EA000CD5BDB4F888380915A06C82FD0E0C701D5
:103EB000865A9F4F0E94EC0A90E00E94AA1CCB5B9E
:103EC000DB4F888300915A0610E0C70182569F4F4E
:103ED0000E94EC0AF801ED5FFB4F882319F0808106
:103EE000806802C080818F77808380915A06C82FB6
:103EF000D0E0C70180569F4F0E94EC0AC95BDB4FA0
:103F0000888380915A06C82FD0E0C7018E559F4FF5
:103F10000E94EC0A90E00E94AA1CC75BDB4F8883DA
:103F200000915A0610E0C7018E599F4F0E94EC0A7B
:103F3000F801EB5FFB4F882319F08081816002C09C
:103F400080818E7F808380915A06C82FD0E0C70180
:103F50008C599F4F0E94EC0AC55BDB4F8883809190
:103F60005A06C82FD0E0C7018A599F4F0E94EC0A19
:103F700090E00E94AA1CC35BDB4F888300915A0625
:103F800010E0C70182599F4F0E94EC0AF801EB5FD5
:103F9000FB4F882319F08081846002C080818B7F71
:103FA000808380915A06C82FD0E0C70180599F4F67
:103FB0000E94EC0AC15BDB4F888380915A06C82FB0
:103FC000D0E0C7018E589F4F0E94EC0A90E00E94FB
:103FD000AA1CCF5ADB4F888300915A0610E0C70114
:103FE00084579F4F0E94EC0AF801EB5FFB4F882338
:103FF00019F08081806802C080818F7780838091F2
:104000005A06C82FD0E0C70182579F4F0E94EC0A82
:10401000CD5ADB4F888380915A06C82FD0E0C70164
:1040200080579F4F0E94EC0A90E00E94AA1CCB5A36
:10403000DB4F888300915A0610E0C7018E569F4FD0
:104040000E94EC0AF801EB5FFB4F882319F0808196
:10405000826002C080818D7F808380915A06C82F44
:10406000D0E0C7018C569F4F0E94EC0AC55ADB4F27
:10407000888380915A06C82FD0E0C7018A569F4F87
:104080000E94EC0A90E00E94AA1CC35ADB4F88836E
:1040900000915A0610E0C7018C589F4F0E94EC0A0D
:1040A000F801EB5FFB4F882319F08081886002C024
:1040B0008081877F808380915A06C82FD0E0C70116
:1040C0008A589F4F0E94EC0AC95ADB4F888380911F
:1040D0005A06C82FD0E0C70188589F4F0E94EC0AAB
:1040E00090E00E94AA1CC75ADB4F888300915A06B1
:1040F00010E0C70186589F4F0E94EC0AF801EB5F61
:10410000FB4F882319F08081806102C080818F7EFF
:10411000808380915A06C82FD0E0C70184589F4FF2
:104120000E94EC0AC15ADB4F888380915A06C82F3F
:10413000D0E0C70182589F4F0E94EC0A90E00E9495
:10414000AA1CCF59DB4F888300915A0610E0C701A3
:1041500080589F4F0E94EC0AF801EB5FFB4F8823C9
:1041600019F08081806202C080818F7D8083809180
:104170005A06C82FD0E0C7018E579F4F0E94EC0A05
:10418000CD59DB4F888380915A06C82FD0E0C701F4
:104190008C579F4F0E94EC0A90E00E94AA1CCB59BA
:1041A000DB4F888300915A0610E0C7018A579F4F62
:1041B0000E94EC0AF801EB5FFB4F882319F0808125
:1041C000806402C080818F7B808380915A06C82FD3
:1041D000D0E0C70188579F4F0E94EC0AC959DB4FB6
:1041E000888380915A06C82FD0E0C70186579F4F19
:1041F0000E94EC0A90E00E94AA1CC759DB4F8883FA
:1042000000915A0610E0C7018C559F4F0E94EC0A9E
:10421000F801E95FFB4F882319F08081816002C0BB
:1042200080818E7F808380915A06C82FD0E0C7019D
:104230008A559F4F0E94EC0AC559DB4F88838091B5
:104240005A06C82FD0E0C70188559F4F0E94EC0A3C
:1042500090E00E94AA1CC359DB4F888300915A0644
:1042600010E0C70180559F4F0E94EC0AF801E95FFA
:10427000FB4F882319F08081846002C080818B7F8E
:10428000808380915A06C82FD0E0C7018E549F4F7B
:104290000E94EC0AC159DB4F888380915A06C82FCF
:1042A000D0E0C7018C549F4F0E94EC0A90E00E941E
:1042B000AA1CCF58DB4F888300915A0610E0C70133
:1042C0008A549F4F0E94EC0AF801E95FFB4F882354
:1042D00019F08081886002C08081877F808380910F
:1042E0005A06C82FD0E0C70188549F4F0E94EC0A9D
:1042F000CD58DB4F888380915A06C82FD0E0C70184
:1043000086549F4F0E94EC0A90E00E94AA1CCB5852
:10431000DB4F888300915A0610E0C70184549F4FF9
:104320000E94EC0AF801E95FFB4F882319F08081B5
:10433000806102C080818F7E808380915A06C82F61
:10434000D0E0C70182549F4F0E94EC0AC958DB4F4E
:10435000888380915A06C82FD0E0C70180549F4FB0
:104360000E94EC0A90E00E94AA1CC758DB4F888389
:1043700000915A0610E0C701845A9F4F0E94EC0A30
:10438000F801E95FFB4F882319F08081806402C047
:1043900080818F7B808380915A06C82FD0E0C7012F
:1043A000825A9F4F0E94EC0AC558DB4F8883809148
:1043B0005A06C82FD0E0C701805A9F4F0E94EC0ACE
:1043C00090E00E94AA1CC358DB4F888300915A06D4
:1043D00010E0C70180529F4F0E94EC0AF801E75F8E
:1043E000FB4F882319F08081846002C080818B7F1D
:1043F000808380915A06C82FD0E0C7018E519F4F0D
:104400000E94EC0AC158DB4F888380915A06C82F5E
:10441000D0E0C7018C519F4F0E94EC0A90E00E94AF
:10442000AA1CCF57DB4F888300915A0610E0C701C2
:104430008C529F4F0E94EC0AF801E75FFB4F8823E4
:1044400019F08081826002C080818D7F808380919D
:104450005A06C82FD0E0C7018A529F4F0E94EC0A2B
:10446000CD57DB4F888380915A06C82FD0E0C70113
:1044700088529F4F0E94EC0A90E00E94AA1CCB57E2
:10448000DB4F8883DF91CF911F910F91FF90EF90C9
:1044900008954F925F927F928F929F92AF92BF92B8
:1044A000CF92DF92EF92FF920F931F93DF93CF9300
:1044B000CDB7DEB7C854D0400FB6F894DEBF0FBEFC
:1044C000CDBF04EA14E0C8010E949505C80166E06A
:1044D00049E00E947004C8010E94480500D000D045
:1044E000EDB7FEB71283018381E092E0948383836A
:1044F0000E94782A0F900F900F900F90C8010E9491
:104500002C0500D000D007E814E0EDB7FEB7128309
:10451000018381EF91E0948383830E94782A56EE91
:10452000452E51E0552EEE24FF24CC24DD240F909F
:104530000F900F900F90702E012F49E0A42EB12CF8
:10454000AC0EBD1E4E010894811C911C87E894E0BE
:104550000E942C2B982F8D3031F08D30DCF1805360
:104560008230C0F530C01830A1F59981892F805371
:10457000823078F5913311F490E801C090E08A819F
:10458000813309F4905C8B81813309F4905E8C81D6
:10459000813309F4905F8D81813309F4985F8E81B6
:1045A000813309F49C5F8F81813309F49E5F888594
:1045B000813309F49F5FF501EE0DFF1D9083089490
:1045C000E11CF11C06C0F401E10FF11D90831F5F97
:1045D00001C010E0F0E4EF16F104C9F484EA94E0BD
:1045E000B601A5010E9480040894C11CD11C00D012
:1045F00000D0EDB7FEB771820283548243820E94DD
:10460000782AEE24FF240F900F900F900F90FFEF69
:10461000CF16D10409F00CF499CFC85BDF4F0FB669
:10462000F894DEBF0FBECDBFCF91DF911F910F91E8
:10463000FF90EF90DF90CF90BF90AF909F908F90C2
:104640007F905F904F900895DF92EF92FF920F93CB
:104650001F93DF93CF93CDB7DEB72A970FB6F894A9
:10466000DEBF0FBECDBF73E0E72EF12CEC0EFD1EBA
:1046700063E0D62E21C40E94223260527E448040E4
:104680009040C8F40E9422326958734180409040A3
:1046900090F01A3011F01D3031F4809123068F5FB5
:1046A0008093230602C01092230680912306833054
:1046B00011F40E944922812F69E175E00E94F206FF
:1046C000882311F400E0F2C380911D0590911E052E
:1046D000A0911F05B0912005863E46EA940746E268
:1046E000A4074DE7B40709F4A0C2873E56EA950730
:1046F00056E2A5075DE7B50708F0F8C08832EEE599
:104700009E07E2EDAE07E4E2BE0709F439C2893242
:10471000FEE59F07F2EDAF07F4E2BF0708F073C0B4
:1047200080352FED92072DEEA20728E1B20709F49C
:1047300079C381353FED93073DEEA30738E1B30719
:1047400088F584304AE9940747EDA4074EE0B407A2
:1047500009F416C285305AE9950757EDA5075EE0C2
:10476000B50780F48E3FEBEC9E07E7ECAE07E9E07F
:10477000BE0709F482C386519A4AA743BB4009F099
:104780008BC3FEC1823923EA92072CEEA20724E1F3
:10479000B20709F4F5C188599C42AA41B64109F013
:1047A0007BC3F7C184344BED940740E7A4074DE188
:1047B000B40709F462C385345BED950750E7A5079C
:1047C0005DE1B50780F48E3CE8E49E07E7E5AE07BF
:1047D000EAE1BE0709F429C284579B4EAA47BB41B0
:1047E00009F05AC3CDC1823D22EC920722E8A2070C
:1047F0002EE1B20709F4CDC18C5A9A4CA64EB042B4
:1048000009F04AC33AC3883546EB94074DEFA40735
:104810004AE4B40709F4E8C2893556EB95075DEF21
:10482000A5075AE4B50788F5863EE5ED9E07EAED53
:10483000AE07E3E3BE0709F451C1873EF5ED9F07DC
:10484000FAEDAF07F3E3BF0780F48E3729EA92074A
:104850002BE5A20726E2B20709F49BC182559342D9
:10486000A649B64209F018C36FC2883F4CEA9407C4
:104870004EEEA40744E3B40709F4FFC2865A9E40F3
:10488000A241B84409F008C398C28036EBED9E07F8
:10489000EBE3AE07EEE6BE0709F472C18136FBED2D
:1048A0009F07FBE3AF07FEE6BF0780F4823E25E5E6
:1048B00092072CE9A20726E6B20709F4A5C28C5E8E
:1048C0009943A647BB4609F0E7C2D7C28A3B47ECEB
:1048D000940741E2A40744E7B40709F4FFC08A57EC
:1048E000974CA94DBB4709F0D7C2C7C28C36E8E642
:1048F0009E07E3E4AE07E2ECBE0709F406C28D367C
:10490000F8E69F07F3E4AF07F2ECBF0708F073C0C7
:104910008A3726EF920721EFA2072DE9B20709F4A3
:1049200084C18B3736EF930731EFA3073DE9B30717
:1049300088F58C3845E8940747EAA40748E9B407A6
:1049400009F473C18D3855E8950757EAA50758E96A
:10495000B50780F48634E3E09E07E2ECAE07E5E8B5
:10496000BE0709F491C282559A4EA048BA4809F090
:1049700093C206C18A362EE2920722E6A20729E9EF
:10498000B20709F41AC28E579241AA46BB4909F0F0
:1049900083C2F6C08A3847EF940747ECA40748EB78
:1049A000B40709F4F6C08B3857EF950757ECA50705
:1049B00058EBB50780F48E3FE6EB9E07E9E2AE07C1
:1049C000E5EABE0709F431C180529E44A94AB14BC1
:1049D00009F062C219C2843A20E092072BE9A207CB
:1049E0002AEBB20709F449C28A5B9448A542BE4B40
:1049F00009F052C209C2843649ED940740EEA4077B
:104A000047EDB40709F46AC0853659ED950750EEB5
:104A1000A50757EDB50788F58435EDE29E07EFEF62
:104A2000AE07E5ECBE0709F4ABC08535FDE29F0794
:104A3000FFEFAF07F5ECBF0780F4803824E792075B
:104A400020E1A20724ECB20709F4A3C086589B43D7
:104A5000A04AB44C09F020C2D7C188324FE994076C
:104A600040E0A40747ECB40709F45FC186599543B9
:104A7000A840B24D09F010C267C18E34EDE59E0723
:104A8000EEE3AE07E3EEBE0709F47AC08F34FDE52E
:104A90009F07FEE3AF07F3EEBF0780F4843727E3F9
:104AA000920724EDA2072EEDB20709F4ADC1865B93
:104AB0009342A34AB24E09F0EFC1B7C0823940E732
:104AC000940746E8A4074BEFB40709F4D6C1825F08
:104AD0009D4EA442BD4F09F0DFC19FC10E9422320A
:104AE0006093C8047093C9048093CA049093CB0464
:104AF000D092C70489E195E060E170E00E94C608A9
:104B00000E944F357093CD046093CC0489E195E009
:104B100064E170E00E94C6080E944F357093CF0494
:104B20006093CE0489E195E068E170E00E94C608D8
:104B30000E944F358B017093D1046093D004609133
:104B4000D2047091D3048091D4049091D50420E0D4
:104B500030E040E050E00E94E034882379F4B8016E
:104B6000882777FD8095982F0E9482356093D60420
:104B70007093D7048093D8049093D90401E08DC139
:104B8000809123058093DA04809124058093DB04CF
:104B900083C189E195E060E070E00E94C60820E0F2
:104BA00030E048EC52E40E94B5360E944F357093D5
:104BB000DD046093DC04693C710520F01092DD0493
:104BC0001092DC0480913D0590913E059093DF04A6
:104BD0008093DE0480913F05909140059093E1041D
:104BE0008093E00480914305909144059093A40242
:104BF0008093A30280914705909148059093A60267
:104C00008093A5028091490590914A059093A8024E
:104C10008093A70280914B0590914C059A838983DC
:104C20009093AA028093A90237C1609123057091E5
:104C3000240580912505909126050E94823520E863
:104C400036E948E15BE40E94E7346093D204709354
:104C5000D3048093D4049093D50460912705709178
:104C600028058091290590912A05D7016C9311960A
:104C70007C93119712968C93129713969C930E9493
:104C8000823520E836E948E15BE40E94E73460932E
:104C9000E2047093E3048093E4049093E50480912C
:104CA00048058093E6048091470584300CF083E04A
:104CB0008093E70489E195E060E170E00E94C60816
:104CC0006093D6047093D7048093D8049093D9044A
:104CD00089E195E068E070E00E94C6086093E8040E
:104CE0007093E9048093EA049093EB0489E195E0E2
:104CF00064E170E00E94C6086093EC047093ED04D8
:104D00008093EE049093EF04C7C089E195E068E0DA
:104D100070E00E94C60890586093F0047093F1040C
:104D20008093F2049093F304B7C089E195E060E0CA
:104D300070E00E94C6086093F4047093F5048093B9
:104D4000F6049093F704A8C089E195E060E070E074
:104D50000E94C6086093F8047093F9048093FA04E3
:104D60009093FB0489E195E064E070E00E94C6083E
:104D700020E030E048EC52E40E94B5360E944F3506
:104D80007093FD046093FC0489E195E064E170E0B8
:104D90000E94C6080E944F357093FF046093FE0482
:104DA00089E195E068E170E00E94C6080E944F35F5
:104DB00070930105609300056FC089E195E064E0A0
:104DC00070E00E94C6080E944F35882777FD8095C5
:104DD000982F0E948235609302057093030580939B
:104DE00004059093050558C089E195E068E070E0FE
:104DF0000E94C6080E944F35709561957F4F709351
:104E000007056093060548C08091830580930805D7
:104E100080918405809309053FC08091230580938C
:104E20000A053AC089E195E060E070E00E94C6089A
:104E300060930B0570930C0580930D0590930E0500
:104E400089E195E064E070E00E94C60860930F0578
:104E500070931005809311059093120589E195E0F8
:104E600068E070E00E94C608609313057093140513
:104E700080931505909316050FC080912F058093A0
:104E800017058091340506C0809130058093170581
:104E9000809135058093180500E080911A058232D3
:104EA00029F489E195E063E20E94DE098EEB90E04F
:104EB0000E948932002331F587E894E00E94FC2AA1
:104EC00018161906F4F487E894E00E942C2B182F8A
:104ED0008091C704882309F0EECBCDCB1092C70494
:104EE00001E0802F90E02A960FB6F894DEBF0FBE47
:104EF000CDBFCF91DF911F910F91FF90EF90DF9089
:104F0000089500E02091C8043091C9044091CA047A
:104F10005091CB04205F384D4F4F5F4F2F83388720
:104F200049875A870E9422322F81388549855A85C0
:104F3000261737074807590788F2D3CFEF92FF9219
:104F40000F931F9380915806882351F081E00E94AF
:104F5000BE3364E070E00E94EF37609328063CC0E7
:104F600081E00E94BE33AA2797FDA095BA2FBC010D
:104F7000CD010E9482352DEC3CEC4CE45EE30E94B6
:104F8000B53620E030E040E85EE30E94B5367B01B4
:104F90008C016091280670E0882777FD8095982F16
:104FA0000E9482352DEC3CEC4CE45FE30E94B53668
:104FB0009B01AC01C801B7010E941A340E9454350C
:104FC00020917306621730F030917206262F361743
:104FD00008F4232F209328061F910F91FF90EF9044
:104FE000089583E00E94BB3308951F93CF93DF930E
:104FF00085E090E06CE070E00E94231668EE73E0BC
:1050000080E090E00E94303287E894E00E94792BA3
:10501000C0E0D0E010E0CE016DE171E00E94EF371A
:10502000892BA9F41F5E84EA94E0612F4CE00E9472
:10503000700484EA94E00E94480584EA94E06EEEED
:105040000E94780584EA94E00E942C05105161E0EA
:1050500070E080E090E00E943032219687E0C13D10
:10506000D807C9F6DF91CF911F91089586E061E0DE
:105070000E94673308950F931F9386E061E00E94BA
:10508000283307E814E0C80140E051EE60E070E02A
:105090000E949A2A1093A3060093A2060E94362823
:1050A00084EA94E00E94CE050E94A11C64EF71E0A6
:1050B00080E090E00E94303283EF93E00E94EC0A9F
:1050C000813011F00E94FD0C0E945D0A10925A0678
:1050D00007C00E94BF1C80915A068F5F80935A06BA
:1050E00080915A068230A8F310925A060E94F52742
:1050F0000E94F12786EB94E06CE07AE224E630E04F
:1051000040E050E000E00E944D3184EA94E00E94CB
:10511000950586EB94E00E94B3311F910F9108959D
:105120002F923F924F925F926F927F928F929F92B7
:10513000AF92BF92CF92DF92EF92FF920F931F93A5
:10514000DF93CF9300D000D0CDB7DEB78091560665
:10515000882309F4E1C0E0907B06F0907C06009182
:105160007D0610917E06C801B7019F7725E33AEFCF
:105170004EE85CE30E94B5360E94E43469837A838A
:105180008B839C83C801B7012091D2043091D30452
:105190004091D4045091D5040E9419341B012C0174
:1051A0009F7720EC3BE649ED57E40E94B5365B0162
:1051B0006C0160917F0670918006809181069091CC
:1051C00082062091E2043091E3044091E40450917E
:1051D000E5040E9419343B014C019F7720EC3BE62B
:1051E00049ED57E40E94B53629813A814B815C81B3
:1051F0000E94B5367B018C01C601B501A60195015F
:105200000E94B5365B016C01C801B701A801970186
:105210000E94B5369B01AC01C601B5010E941A344B
:105220000E943C370E944F356093490670934A06AE
:1052300080934B0690934C0660E070E080E89FE31B
:1052400029813A814B815C810E94E7349B01AC014A
:10525000C201B1010E94B53697FA909497F89094E4
:10526000A40193010E948D3420EE3EE245E652E413
:105270000E94B53620E030E044EB52E40E941A343C
:105280000E944F359B01AC0197FF04C028593E4F47
:105290004F4F5F4FCA01B901645B7040804090403E
:1052A00097FF06C0CA01B9016C547F4F8F4F9F4FC3
:1052B0000E9482352091D6043091D7044091D804C1
:1052C0005091D9040E9419340E944F3597FF04C0B1
:1052D00068597E4F8F4F9F4F0E94823520E030E00B
:1052E00044EB53E40E94E73420E030E040E851E42E
:1052F0000E94B5360E94183720E030E040E85FE3B6
:105300000E941A340E94543560934806613108F4B3
:105310006CC01092480669C08091E704823008F49E
:1053200064C08091E604853008F45FC0A0908306D5
:105330008DE18A1508F459C0E090E804F090E90482
:105340000091EA041091EB04609184067091850647
:105350008091860690918706A80197010E941934D2
:105360009F7720E030E040E05FE30E94AA36181605
:105370005CF410928306E0928406F0928506009316
:1053800086061093870631C08A2D8F5F809383062F
:105390008E3159F58091D2049091D304A091D40418
:1053A000B091D50480937B0690937C06A0937D06F4
:1053B000B0937E068091E2049091E304A091E4040E
:1053C000B091E50480937F0690938006A0938106B8
:1053D000B0938206E0928806F092890600938A06CE
:1053E00010938B0681E0809356060F900F900F90DC
:1053F0000F90CF91DF911F910F91FF90EF90DF9071
:10540000CF90BF90AF909F908F907F906F905F9064
:105410004F903F902F900895CF92DF92EF92FF929E
:105420000F931F930E949E2780912806282F30E01B
:105430003093AC022093AB0280915806882359F533
:105440000091730610E0201B310BB901882777FD0E
:105450008095982F0E9482356B017C0160917206C5
:1054600070E0601B710B882777FD8095982F0E9454
:1054700082359B01AC01C701B6010E94E73420E0F0
:1054800030E048EC52E40E94B5360E944F357093EC
:10549000AC026093AB028091AB029091AC028D594B
:1054A0009F4F34F48DE99FEF9093AC028093AB0251
:1054B0000E944F080E94F20A84EA94E00E94902819
:1054C0000E94701A1F910F91FF90EF90DF90CF9084
:1054D00008950E942423892B19F00E940C2A089514
:1054E00086EB94E00E949B3108958FEF9FE708952B
:1054F000DF93CF93CDB7DEB7FE0139968D819E81C4
:1055000061E04F8158859F010E94192DCF91DF9155
:105510000895DF93CF93CDB7DEB7FE0139968D8125
:105520009E8160E04F8158859F010E94192DCF9187
:10553000DF9108950F931F93DC01ED91FC91028898
:10554000F389E02D20E030E000E010E009951F91A4
:105550000F9108958F92AF92CF92EF92FF920F9397
:105560001F93DF93CF93CDB7DEB7FC011382128276
:1055700088EE93E0A0E0B0E084839583A683B783B0
:105580008AEE93E091838083558744873787268707
:10559000118B008BF38AE28AC48AA58A868A70E01E
:1055A000CB0123E0880F991F2A95E1F79C01205732
:1055B000394F308F278B8856994F928F818F81E09A
:1055C00090E002C0880F991F6A95E2F72091A0062B
:1055D000282B2093A006CF0140E051EE60E070E060
:1055E0000E949A2ACF91DF911F910F91FF90EF9027
:1055F000CF90AF908F900895FC01838D882319F48C
:105600002FEF3FEF0DC00788F08DE02D2081318115
:1056100082819381281B390B84819581282339232A
:10562000C9010895FC01838D882319F42FEF3FEF02
:1056300011C0018CF28DE02D208131818281938116
:10564000281B390B20953095848195812823392397
:105650002F5F3F4FC9010895FC01838D882361F0BE
:10566000A789B08D2D913C91119712968D919C91A7
:1056700013972817390721F44FEF5FEFCA010895F8
:1056800012968D919C9113971696ED91FC91179718
:10569000E80FF91F408112968D919C911397019606
:1056A00014962D913C9115978223932313969C93E6
:1056B0008E93129750E0E2CFFC01838D882351F046
:1056C0000788F08DE02D2081318182819381281718
:1056D000390721F42FEF3FEFC901089582819381AB
:1056E0000680F781E02DE80FF91F8081282F30E038
:1056F000F3CFDC015796ED91FC915897828193810D
:10570000918380835996ED91FC915A978081918184
:10571000938382830895DC015B968C915B97882349
:10572000A9F15996ED91FC915A97208131812F5F13
:105730003F4F84819581282339235C968C915C9717
:10574000882329F08281938128173907F9F0828113
:10575000938128173907D9F3808191810680F781D9
:10576000E02DE80FF91F60835996ED91FC915A974F
:10577000318320835296ED91FC9153978081569608
:105780009C91892B808321E030E002C020E030E052
:10579000C9010895CF93DF93EC011B821A828A819D
:1057A0009B81998388831D821C828E819F810097B3
:1057B00021F00E94C2031F821E82DF91CF910895C3
:1057C0000F931F938C01DC015296ED91FC9153973E
:1057D000208156968C91569755969C915597892B7A
:1057E00080958223808357968D919C9158970E9433
:1057F000CA2BF801818D928D0E94CA2BD8015B962D
:105800001C921F910F9108950F931F93CF93DF93D5
:105810008C01FC01138212828281938191838083A7
:1058200041E0A1E0B0E001C04F5FFD01042E02C0E5
:10583000EE0FFF1F0A94E2F79B0182E061307807C8
:1058400010F020E032E0E217F30770F3C1E0D0E09F
:1058500002C0CC0FDD1F4A95E2F72197F80126819F
:1058600037812115310541F0848195818C179D0781
:1058700089F0C9010E94C203F801D583C483CE0117
:1058800001960E9418039C01F8019783868380E0AB
:10589000232B09F081E0DF91CF911F910F910895A3
:1058A000AF92BF92CF92DF92EF92FF920F931F932E
:1058B000CF93DF937C015A016B01E901DC015B9618
:1058C0008C915B978823F1F02115310539F45796B7
:1058D000ED91FC915897C481D58121960115110550
:1058E00049F4D7015996ED91FC915A97048115819D
:1058F0000F5F1F4FD701ED91FC910088F189E02DDA
:10590000C7010995F7018789908D209711F4C0E8A8
:10591000D0E0BE010E94042C882381F0D701599663
:105920008D919C915A970115110511F400E110E039
:10593000B8010E94042C882309F04DC0D701ED91D5
:10594000FC910088F189E02DC701099567C0D70156
:105950005096ED91FC915197B0E0AB16B1EEBB06BD
:10596000B0E0CB06B0E0DB0609F454C081E090E083
:10597000D70154960C9002C0880F991F0A94E2F741
:10598000808360E079E08DE390E0A60195010E94BC
:1059900024382150304040405040CA01B90122E033
:1059A00030E040E050E00E942438D7011C96ED9191
:1059B000FC911D9730831E96ED91FC911F972083DB
:1059C000D7015296ED91FC915397808155969C9109
:1059D000892B808323C0D7015996ED91FC915A976A
:1059E0001382128282819381918380835796ED91F5
:1059F000FC915897138212828281938191838083D4
:105A000081E05B968C931A141B041C041D040CF497
:105A10009ECFD6CF108220E130E0C7CFDF91CF916B
:105A20001F910F91FF90EF90DF90CF90BF90AF90BC
:105A300008952F923F924F925F926F927F928F9232
:105A40009F92AF92BF92CF92DF92EF92FF920F930D
:105A50001F93DF93CF93CDB7DEB764970FB6F8945B
:105A6000DEBF0FBECDBF3C01688B5A8B498B6901ED
:105A70001C01AE014F5F5F4F5C8B4B8BE989FA894C
:105A8000488940FD659140FF6191FA8BE98B66235F
:105A900009F4D7C3653249F440FD859140FF8191F7
:105AA000FA8BE98B8532B1F40CC06A3051F4D30122
:105AB000ED91FC910190F081E02DC1016DE009951F
:105AC0006AE0D301ED91FC910190F081E02DC101DC
:105AD0000995D4CF982F10E0882499241032B0F47F
:105AE0009B3269F09C3228F4903251F0933271F479
:105AF0000BC09D3239F0903349F4116028C0126018
:105B0000146025C0186023C0106121C017FD2BC090
:105B1000892F80538A3078F416FF06C0BAE09B9E26
:105B2000902C1124980E13C0EAE08E9E802C112434
:105B3000880E10620CC09E3221F416FD82C31064E0
:105B400006C09C3611F4106802C0983661F4E989E9
:105B5000FA89488940FD959140FF9191FA8BE98B34
:105B6000992309F0BBCF892F8554833020F4812FEE
:105B70008061905E07C0892F8556833008F0E6C1AA
:105B8000812F8F7E86FD02C076E0972E6FE3F62E82
:105B9000F822953619F450E4F52A07C0963619F420
:105BA00080E8F82A02C091109A94F7FE0BC09BE39C
:105BB000991520F427E05CE3B52E0DC0B92CB39401
:105BC00027E009C0A7E0A91520F447E0942E27E0BC
:105BD00001C0292DBB24F6013496FD87EC87D60140
:105BE0006D917D918D919C91AE014F5F5F4F0B2D1B
:105BF0000E9440026C010981E02FF0E0FF87EE87F0
:105C000000FF05C0FE85F3FD02C01DE209C0F1FEE4
:105C100002C01BE205C0F2FC02C010E001C010E2AD
:105C20008E859F858C709070892B09F444C0112358
:105C300011F483E001C084E0881510F088240EC0C0
:105C4000881AF3FC0BC0D301ED91FC910190F08117
:105C5000E02DC10160E209958A94A9F7112349F06A
:105C6000D301ED91FC910190F081E02DC101612FF4
:105C70000995BE85B3FF03C00AE013E012C00EE031
:105C800013E00FC0E114F10409F06052D301ED916B
:105C9000FC910190F081E02DC10109950F5F1F4F2C
:105CA00005C0EF2CFF24B0E1EB22FF24F801649142
:105CB000662341F748C1F7FE13C0BC0CFE85F4FF14
:105CC00004C08A81813309F4BA941B141CF0BB24EC
:105CD000B3942DC048E04B1550F538E0B32E27C0E3
:105CE000F6FC25C0892D90E08C159D054CF05CEFED
:105CF000C5165FEFD50624F080E8F82A01C09A9413
:105D0000992049F0E2E0F0E0EC0FFD1FE90DF11DF4
:105D100080818033A1F3F7FE0AC0B92CB394892D9A
:105D200090E0C816D90614F0992401C09C18F7FC1D
:105D300003C025E030E009C01C141D041CF021E064
:105D400030E003C096012F5F3F4F112311F02F5F0A
:105D50003F4F992029F0892D90E00196280F391F97
:105D6000882D90E02817390714F0882401C0821A82
:105D70004F2C5524C20189709070892B59F00CC0AA
:105D8000D301ED91FC910190F081E02DC10160E221
:105D900009958A948820A1F7112349F0D301ED9148
:105DA000FC910190F081E02DC101612F099543FE26
:105DB0000BC00CC0D301ED91FC910190F081E02D5E
:105DC000C10160E309958A948820A1F7F7FE51C0CC
:105DD0008601D7FE02C000E010E076010894E11CC5
:105DE000F11CE01AF10AE1E0F0E0EC0FFD1FEE0E0D
:105DF000FF1E26014B185108892D90E0AA24BB24D0
:105E0000A81AB90AFFEF0F3F1F0749F4D301ED911C
:105E1000FC910190F081E02DC1016EE20995C01660
:105E2000D10634F0401651061CF4F701608101C020
:105E300060E3015010400894E11CF11C0A151B0599
:105E40004CF0D301ED91FC910190F081E02DC10166
:105E50000995D8CF0C151D0541F48A81863320F4AD
:105E6000853319F4BE85B4FF61E3D301ED91FC9154
:105E700065C06A81613309F00F7ED301ED91FC9119
:105E80000190F081E02DC10109959920E1F0D30145
:105E9000ED91FC910190F081E02DC1016EE2099538
:105EA00012E0E1E0F0E0EC0FFD1FE10FF11D608179
:105EB0001F5FD301ED91FC910190F081E02DC101B4
:105EC00009959A9471F7D301ED91FC910190F081BD
:105ED000E02D44FC02C065E601C065E4C1010995FE
:105EE000D7FC05C0C114D10441F404FF06C0D0940E
:105EF000C194D108D3946DE201C06BE2D301ED915E
:105F0000FC910190F081E02DC101099560E305C08D
:105F10006F5FE6EFFFEFCE0EDF1EFAE0CF16D10483
:105F2000BCF7D301ED91FC910190F081E02DC1010E
:105F30000995D301ED91FC916C2D605D0190F0818C
:105F4000E02DC1010995CC84DD8478C1933631F010
:105F5000933799F0933509F061C023C0F601808131
:105F600089835E010894A11CB11C42E050E0C40E7C
:105F7000D51E21E0E22EF12C12C0D601AD90BC90CE
:105F800016FD03C06FEF7FEF02C0692D70E0E2E005
:105F9000F0E0CE0EDF1EC5010E9425047C011F77B4
:105FA00013C0D601AD90BC9016FD03C06FEF7FEF1C
:105FB00002C0692D70E0E2E0F0E0CE0EDF1EC50108
:105FC0000E941A047C01106813FF0BC023C0D30188
:105FD000ED91FC910190F081E02DC10160E2099505
:105FE0008A94882D90E0E816F90688F313C0F5012D
:105FF00017FD659117FF61915F01D301ED91FC9150
:106000000190F081E02DC101099581108A940894D6
:10601000E108F108E114F10451F710C1943611F0D0
:10602000993699F517FF0AC0F60120813181428126
:10603000538184E090E0C80ED91E0CC0D6018D912A
:106040009C919C01442737FD4095542FE2E0F0E0FD
:10605000CE0EDF1E9FE6F92EF12257FF09C05095A4
:106060004095309521953F4F4F4F5F4FF0E8FF2A05
:10607000CA01B901AE014F5F5F4F2AE030E00E94D4
:10608000E201E82E4B89E41A41C0953721F41F7EC6
:106090002AE030E01CC0197F9F3661F0903720F471
:1060A000983509F0CEC00FC0903739F0983709F015
:1060B000C8C004C028E030E00AC0106114FD1460BC
:1060C00020E130E004C014FD166020E132E017FF4B
:1060D00008C0D6016D917D918D919C91E4E0F0E036
:1060E00008C0D6018D919C91BC0180E090E0E2E077
:1060F000F0E0CE0EDF1EAE014F5F5F4F0E94E20167
:10610000E82EFB89EF1A8FE7F82EF122F6FE0BC07E
:106110004EEFF422E91438F4F4FE07C0F2FC05C097
:106120005FEEF52202C01E2D01C0192DF4FE0DC038
:10613000FE01EE0DF11D8081803319F489EEF82205
:1061400008C01F5FF2FE05C003C08F2D867809F0DE
:106150001F5F0F2DF3FC18C0F0FE13C0181510F0D0
:106160009E2C0FC09E2C980C911A182D0AC0D3019A
:10617000ED91FC910190F081E02DC10160E2099563
:106180001F5F1815A0F304C0181510F4811A01C080
:10619000882404FF17C0D301ED91FC910190F08198
:1061A000E02DC10160E3099502FF29C0D301ED9103
:1061B000FC910190F081E02D01FD02C068E712C062
:1061C00068E510C0802F8678D1F001FF02C06BE235
:1061D00001C060E2F7FC6DE2D301ED91FC9101900A
:1061E000F081E02DC10109950AC0D301ED91FC9128
:1061F0000190F081E02DC10160E309959A94E914C2
:10620000A0F3EA94D301ED91FC91A1E0B0E0AC0FD2
:10621000BD1FAE0DB11D0190F081E02DC1016C914B
:106220000995EE2071F70AC0D301ED91FC91019020
:10623000F081E02DC10160E209958A948820A1F7E0
:106240001DCC64960FB6F894DEBF0FBECDBFCF91C4
:10625000DF911F910F91FF90EF90DF90CF90BF9053
:10626000AF909F908F907F906F905F904F903F90F6
:106270002F900895F999FECF72BD61BDF89A80B54F
:106280000895F999FECF1FBA72BD61BD40BD0FB62A
:10629000F894FA9AF99A0FBE08950F93FC016115CC
:1062A000710511F480E011C021833283438354834C
:1062B000728761870170000F000F000F8081877F58
:1062C000802B82608B7F808381E00F910895CF9334
:1062D000DF93EC010E9422329B01AC018D819E81F3
:1062E000AF81B885281739074A075B0728F48881EA
:1062F00084FD02C060E00DC089819A81AB81BC81C0
:10630000820F931FA41FB51F8D839E83AF83B88711
:1063100061E0222757FD2395332744275527922FE5
:1063200091709295907F88818F7E892B8883862FAC
:10633000DF91CF910895CF93DF93EC01888182FFA5
:106340000FC0CE010E946731882351F0E985FA859C
:10635000309709F00995888183FF02C08B7F88837D
:10636000DF91CF910895CF93DF93EC0189859A85D2
:10637000892BE1F089819A81AB81BC810097A105CD
:10638000B105A1F00E94223229813A814B815C81C2
:10639000260F371F481F591F2D833E834F83588771
:1063A000888184608F7E888381E001C080E0DF91F6
:1063B000CF9108951F920F920FB60F9211242F9331
:1063C0003F938F939F93AF93BF938091A806909133
:1063D000A906A091AA06B091AB063091AC06019631
:1063E000A11DB11D232F2D5F2D3720F02D570196B4
:1063F000A11DB11D2093AC068093A8069093A90619
:10640000A093AA06B093AB068091A4069091A5062E
:10641000A091A606B091A7060196A11DB11D80937B
:10642000A4069093A506A093A606B093A706BF91D5
:10643000AF919F918F913F912F910F900FBE0F9031
:106440001F9018958FB7F8942091A8063091A9064F
:106450004091AA065091AB068FBFB901CA010895B9
:106460009B01AC017FB7F8948091A4069091A5069A
:10647000A091A606B091A70666B5A89B05C06F3F80
:1064800019F00196A11DB11D7FBFBA2FA92F982F1A
:106490008827860F911DA11DB11D62E0880F991FED
:1064A000AA1FBB1F6A95D1F7BC012DC0FFB7F89496
:1064B0008091A4069091A506A091A606B091A7068A
:1064C000E6B5A89B05C0EF3F19F00196A11DB11DCF
:1064D000FFBFBA2FA92F982F88278E0F911DA11DBE
:1064E000B11DE2E0880F991FAA1FBB1FEA95D1F7E3
:1064F000861B970B885E9340C8F221503040404085
:10650000504068517C4F211531054105510571F608
:106510000895019739F0880F991F880F991F0297E6
:106520000197F1F70895789484B5826084BD84B5AD
:10653000816084BD85B5826085BD85B5816085BD7E
:10654000EEE6F0E0808181608083E1E8F0E0108297
:10655000808182608083808181608083E0E8F0E0D8
:10656000808181608083E1EBF0E0808184608083C2
:10657000E0EBF0E0808181608083EAE7F0E08081F9
:106580008460808380818260808380818160808359
:106590008081806880831092C10008951F920F92BD
:1065A0000FB60F9211242F933F934F935F936F93E6
:1065B0007F938F939F93AF93BF93EF93FF938091BC
:1065C000AD069091AE06892B29F0E091AD06F091D1
:1065D000AE060995FF91EF91BF91AF919F918F9179
:1065E0007F916F915F914F913F912F910F900FBECF
:1065F0000F901F9018951F920F920FB60F921124B3
:106600002F933F934F935F936F937F938F939F93BA
:10661000AF93BF93EF93FF938091AF069091B00635
:10662000892B29F0E091AF06F091B0060995FF9112
:10663000EF91BF91AF919F918F917F916F915F91FA
:106640004F913F912F910F900FBE0F901F90189573
:10665000CF93DF93482F50E0CA018C5B9C4FFC0125
:106660003491405D5C4FFA018491882369F190E098
:10667000880F991FFC01EE5EFC4FA591B491FC01BF
:10668000E45EFC4FC591D491662351F42FB7F89482
:106690008C91932F909589238C93888189230BC0AB
:1066A000623061F42FB7F8948C91932F90958923E1
:1066B0008C938881832B88832FBF06C09FB7F89463
:1066C0008C91832B8C939FBFDF91CF910895482F9E
:1066D00050E0CA01885A9C4FFC012491CA018C5B8E
:1066E0009C4FFC019491405D5C4FFA01349133233F
:1066F00009F440C0222351F1233071F0243028F4F2
:106700002130A1F0223011F514C02630B1F027302D
:10671000C1F02430D9F404C0809180008F7703C089
:10672000809180008F7D8093800010C084B58F772A
:1067300002C084B58F7D84BD09C08091B0008F7781
:1067400003C08091B0008F7D8093B000E32FF0E014
:10675000EE0FFF1FE45EFC4FA591B4912FB7F894A4
:10676000662321F48C919095892302C08C91892B0A
:106770008C932FBF08958093AF020895982F8E3089
:1067800008F09E5097708091AF028295880F880F15
:10679000807C892B80937C0080917A008064809338
:1067A0007A0080917A0086FDFCCF2091780040919C
:1067B0007900942F80E030E0282B392BC90108950F
:1067C000CF92DF92EF92FF920F931F93CF93DF93BD
:1067D0007C016B018A01C0E0D0E00FC0D6016D9151
:1067E0006D01D701ED91FC910190F081E02DC70181
:1067F0000995C80FD91F015010400115110571F7F7
:10680000CE01DF91CF911F910F91FF90EF90DF901C
:10681000CF900895CF93DF930E9493320E943B283C
:10682000C0E0D0E00E94692A2097E1F30E940000B6
:10683000F9CF5058BB27AA270ED041C201D230F061
:1068400006D220F031F49F3F11F41EF4C0C10EF4C3
:10685000E095E7FBB6C1E92F54D280F3BA1762077F
:1068600073078407950718F071F49EF56CC20EF457
:10687000E0950B2EBA2FA02D0B01B90190010C0150
:10688000CA01A0011124FF27591B99F0593F50F468
:10689000503E68F11A16F040A22F232F342F4427C0
:1068A000585FF3CF469537952795A795F0405395B8
:1068B000C9F77EF41F16BA0B620B730B840BBAF088
:1068C0009150A1F0FF0FBB1F661F771F881FC2F7F3
:1068D0000EC0BA0F621F731F841F48F48795779507
:1068E0006795B795F7959E3F08F0B3CF9395880FBE
:1068F00008F09927EE0F979587950895A1D158F044
:1069000080E891E009F49EEFA2D128F040E851E040
:1069100059F45EEF09C05BC116C2E92FE078F1D1EE
:1069200068F3092E052AC1F32617370748075907C8
:1069300038F00E2E07F8E02569F0E025E0640AC083
:10694000EF6307F8009407FADB01B9019D01DC0150
:10695000CA01AD01EF934AD0B2D10AD05F9155235D
:1069600031F02BED3FE049E450FD49EC63CF089551
:10697000DF93DD27B92FBF7740E85FE316161706D0
:1069800048075B0710F4D92FE9D19F938F937F932A
:106990006F93BCD2E8E6F0E01DD191D12F913F91E9
:1069A0004F915F91EED1DD2349F09058A2EA2AED94
:1069B0003FE049EC5FE3D0785D274DDFDF917FC199
:1069C000DCD008F481E008954AD1E39589C10CD068
:1069D00076C13DD140F034D130F021F45F3F19F061
:1069E000F0C05111B1C1F3C08CD198F39923C9F310
:1069F0005523B1F3951B550BBB27AA2762177307C5
:106A0000840738F09F5F5F4F220F331F441FAA1F78
:106A1000A9F333D00E2E3AF0E0E830D09150504038
:106A2000E695001CCAF729D0FE2F27D0660F771FE6
:106A3000881FBB1F261737074807AB07B0E809F0C8
:106A4000BB0B802DBF01FF2793585F4F2AF09E3F5D
:106A5000510568F0B6C078C15F3FECF3983EDCF3B7
:106A6000869577956795B795F7959F5FC9F7880FD6
:106A7000911D9695879597F90895E1E0660F771F28
:106A8000881FBB1F621773078407BA0720F0621BB9
:106A9000730B840BBA0BEE1F88F7E095089504D0B2
:106AA0006894B11151C1089534D188F09F5790F086
:106AB000B92F9927B751A0F0D1F0660F771F881F23
:106AC000991F1AF0BA95C9F712C0B13081F03BD1C5
:106AD000B1E0089538C1672F782F8827B85F39F063
:106AE000B93FCCF3869577956795B395D9F73EF482
:106AF00090958095709561957F4F8F4F9F4F08952A
:106B0000E89409C097FB3EF4909580957095619547
:106B10007F4F8F4F9F4F9923A9F0F92F96E9BB27FD
:106B20009395F695879577956795B795F111F8CF79
:106B3000FAF4BB0F11F460FF1BC06F5F7F4F8F4FE4
:106B40009F4F16C0882311F096E911C0772321F0DA
:106B50009EE8872F762F05C0662371F096E8862F72
:106B600070E060E02AF09A95660F771F881FDAF7C9
:106B7000880F9695879597F90895990F0008550FF6
:106B8000AA0BE0E8FEEF16161706E807F907C0F0B3
:106B900012161306E407F50798F0621B730B840BBB
:106BA000950B39F40A2661F0232B242B252B21F495
:106BB00008950A2609F4A140A6958FEF811D811D35
:106BC000089597F99F6780E870E060E008959FEF6F
:106BD00080EC0895DF93CF931F930F93FF92EF9272
:106BE000DF927B018C01689405C0DA2EEF01C9D0D9
:106BF000FE01E894A5912591359145915591AEF30B
:106C0000EF0129DEFE019701A801DA9479F7DF9000
:106C1000EF90FF900F911F91CF91DF9108959F9377
:106C20008F937F936F93FF93EF939B01AC019DD064
:106C3000EF91FF91CFDF2F913F914F915F9195C0E1
:106C400000240A941616170618060906089500244B
:106C50000A9412161306140605060895B8CF59D0E3
:106C6000E8F3E894EFEFBB273FE048EC5FE76B3DCC
:106C700073078407950708F1FF279F57B25A6A4D9B
:106C80007F40894CF04032F4BE556542704F8643D8
:106C9000FF4F0894EE1F915030F0BB0F661F771F17
:106CA000881FFF1FEBCF9EE7882332F0BB0F661FC4
:106CB000771F881F9A95C1F79395E09565C1092EB6
:106CC0000394000C11F4882352F0BB0F40F4BF2B47
:106CD00011F460FF04C06F5F7F4F8F4F9F4F089587
:106CE000EF93E0FF06C0A2EA2AED3FE049EC5FEB3C
:106CF000B2DDE5DF0F90039401FC9058E5E9F0E088
:106D00008ECF57FD9058440F551F59F05F3F71F0DB
:106D10004795880F97FB991F61F09F3F79F0879502
:106D20000895121613061406551FF2CF4695F1DF8B
:106D300008C0161617061806991FF1CF869571051B
:106D4000610508940895E894BB2766277727CB014F
:106D500097F9089512DF08F48FEF08959B01AC01B5
:106D600060E070E080E89FE332CE0BD0A8CF68DF10
:106D700028F06DDF18F0952309F023CF28CF1124D8
:106D8000E3CFBFDFA0F3959FD1F3950F50E0551FE0
:106D9000629FF001729FBB27F00DB11D639FAA2770
:106DA000F00DB11DAA1F649F6627B00DA11D661FBF
:106DB000829F2227B00DA11D621F739FB00DA11DE0
:106DC000621F839FA00D611D221F749F3327A00D9A
:106DD000611D231F849F600D211D822F762F6A2F36
:106DE00011249F5750408AF0E1F088234AF0EE0FBB
:106DF000FF1FBB1F661F771F881F91505040A9F7C8
:106E00009E3F510570F0DDCE9FCF5F3FECF3983E83
:106E1000DCF3869577956795B795F795E7959F5F2E
:106E2000C1F7FE2B880F911D9695879597F90895C8
:106E300070DFE0F09E37D8F09639B8F49E3848F409
:106E4000672F782F8827985FF9CF86957795679574
:106E500093959539D0F3B62FB1706B0F711D811DCD
:106E600020F4879577956795939573C08DC06CCF07
:106E700011F40EF4ACCE88C04CDFD0F39923D9F3D3
:106E8000CEF39F57550B87FF8FD056959795B0E05F
:106E900020F4660F771F881FBB1F1F930F930024DA
:106EA0009001A0018001F001A0E80E0F1F1F0A1E33
:106EB000511D601B710B8009B50B48F4600F711FE9
:106EC000801DB51F0E1B1F0B0A0A510907C02E0F8C
:106ED0003F1F4A1F0E0F1F1F0A1E511D660F771FEF
:106EE000881FBB1FA695F795E795F8F606171707B5
:106EF00008065B07211D311D411D0F911F91B9012E
:106F0000842F9158880F9695879508959B01AC0121
:106F10002CCFDF93D92FA3DEE695D7952AED3FE05E
:106F200049E45FE3B33A6207730784079507D7958F
:106F30002AF0A2EA49EC90688EDCC1DEE3EBF0E0D7
:106F40006EDEDD0F0BF00ADFDD0F0BF49058DF91E2
:106F50000895882371F4772321F09850872B762F9A
:106F600007C0662311F499270DC09051862B70E05D
:106F700060E02AF09A95660F771F881FDAF7880F6E
:106F80009695879597F908959F3F49F0915028F479
:106F9000869577956795B7959F5F80389F4F880F47
:106FA0009695879597F9089591505040660F771FF1
:106FB000881FD2F70895AA1BBB1B51E107C0AA1F67
:106FC000BB1FA617B70710F0A61BB70B881F991F8A
:106FD0005A95A9F780959095BC01CD01089597FB2E
:106FE000092E07260AD077FD04D0E5DF06D0002061
:106FF0001AF4709561957F4F0895F6F790958195F5
:107000009F4F0895A1E21A2EAA1BBB1BFD010DC0C4
:10701000AA1FBB1FEE1FFF1FA217B307E407F50748
:1070200020F0A21BB30BE40BF50B661F771F881F24
:10703000991F1A9469F760957095809590959B01BA
:10704000AC01BD01CF01089597FB092E05260ED096
:1070500057FD04D0D7DF0AD0001C38F45095409576
:10706000309521953F4F4F4F5F4F0895F6F790951C
:107070008095709561957F4F8F4F9F4F0895EE0FCC
:0E708000FF1F0590F491E02D0994F894FFCFC6
:10708E002563002563256300256325326925632565
:10709E003032697C256325326925632530326900DB
:1070AE0025632532692563253032690025352E305A
:1070BE0066256300256325312E356625630025631D
:1070CE00253569256300256325352E326625630037
:1070DE006D616E007374310073743200737433001B
:1070EE007374340073743500737436007068200046
:1070FE00636C200076722000686C200061702000A6
:10710E00727462006C616E0070702000706F6900A6
:10711E0061632000006174200025632573002563E0
:10712E0025332E30692563002534692563256300D8
:10713E00256325336925630025737C256325732517
:10714E00630020C0C0C0C0C0C7C0C0C0C0C0200047
:10715E0025342E3066256300256325332E306625B3
:10716E006300256325352E306625630025632531A2
:10717E00312E36667C25632531312E366600256329
:10718E002532690025332E3166256300202020200C
:10719E00202020202020202000202064697361728E
:1071AE006D6564202000206E6F2074656C20636F07
:1071BE006D2000206E6F2067707320666978200046
:1071CE0062617474207761726E696E6700626174B9
:1071DE0074637269746963616C00206261747420F7
:1071EE006572726F722000202072737369206C6F4B
:1071FE00772020006D6167207761726E696E67007F
:10720E006D616720637269746963616C00206D61E2
:10721E006720206572726F7220002573002000B502
:10722E00060000E803E803E803E8039DFF0164019C
:10723E00000000007805E033760479047C047F04B6
:10724E00752A00070E091C1B1215383F36312423F0
:10725E002A2D70777E796C6B6265484F4641545388
:10726E005A5DE0E7EEE9FCFBF2F5D8DFD6D1C4C3F8
:10727E00CACD90979E998C8B8285A8AFA6A1B4B3E8
:10728E00BABDC7C0C9CEDBDCD5D2FFF8F1F6E3E458
:10729E00EDEAB7B0B9BEABACA5A28F888186939448
:1072AE009D9A2720292E3B3C35321F1811160304B8
:1072BE000D0A5750595E4B4C45426F6861667374A8
:1072CE007D7A898E878095929B9CB1B6BFB8ADAA08
:1072DE00A3A4F9FEF7F0E5E2EBECC1C6CFC8DDDA08
:1072EE00D3D4696E676075727B7C51565F584D4A78
:1072FE004344191E171005020B0C21262F283D3A68
:10730E0033344E49404752555C5B7671787F6A6DD7
:10731E0064633E39303722252C2B0601080F1A1DC7
:10732E001413AEA9A0A7B2B5BCBB9691989F8A8D37
:10733E008483DED9D0D7C2C5CCCBE6E1E8EFFAFD27
:10734E00F4F3C2C0C0C1C0C0C1C0C0C4C0C0C1C0BF
:10735E00C0C1C0C0C3C0C0C1C0C0C1C0C0C5C0C014
:10736E00C1C0C0C1C0C0000000008B2BE033FC2A9E
:0E737E002C2B5C2B792B122B9A2AE02B502CF7
:00000001FF
